:020000040800F2
:10000000EA17002425030008A9020008A902000835
:10001000A9020008A9020008A9020008A902000814
:10002000A9020008A9020008A9020008A902000804
:10003000A9020008A9020008A9020008A9020008F4
:10004000A9020008A9020008A9020008A9020008E4
:10029000A9020008A90200080000000000000000F8
:1002A000FFECC2925D7D05C5EFF305801EF0040FE3
:1002B00002D0EFF309818D466A4602F16802EFF33E
:1002C00011832DED108A2DE9FC4F69466C46DFF84D
:1002D00050D000F001FA2146884213D000F16C01A1
:1002E000B1E8F00FB1EC100A91E80C00016821E9C7
:1002F0000C0021ED100A21E9F00FB0E8FC4F90EC62
:10030000108A03E0B1E8FC4FB1EC108A1EF0040F34
:100310000CBF81F3088881F3098883F31188704743
:10032000E002002408B51F4A00211F4B934231D33D
:100330001E4A1F4B1F498B422FD300F01BF9EFF3CE
:10034000148343F0040383F314881B4A1368A2F553
:10035000D67223F04043C2F8AC31136843F4700303
:10036000136000F05DF9BFF34F8FBFF36F8F134A37
:10037000136823F001031360536823F001035360F3
:10038000BFF34F8FBFF36F8F00F03DFC00F008FA12
:1003900000F04CFC43F8041BC8E752F8040F43F884
:1003A000040BC8E7FC140024E00000243CA0000873
:1003B00000000024DC00002434EF00E090EF00E0B7
:1003C000594B82B01A6822F4802242F480321A60BB
:1003D000564A0192019A002A00F39F80019B002B4C
:1003E00040F39980524A5349136823F4706323F011
:1003F0000F0343F0080313600B6823F4E06343F03A
:1004000040030B600B6823F4E06343F480630B60EC
:10041000136823F0700343F040031360936823F0E4
:10042000700343F040039360434B444A283B9A6275
:10043000434A1A63434A9A6302F500321A64424AF5
:10044000DA621A6842F0A8521A601A689201FCD562
:100450001A681001FCD5344A13689900FCD53B4A50
:10046000136843F006031360394B1A6842F44042A4
:100470001A601A689204FCD536490A689004FCD5C3
:1004800035490A6842F002020A6034490A6842F0BB
:1004900001020A601A689204FCD5314B22221A60CC
:1004A000304B1A6822F0070242F003021A601A6801
:1004B00002F03802182AFAD12B482C4A036823F498
:1004C000405343F400530360136823F4407343F430
:1004D00000731360264B196821F4E04141F4805108
:1004E0001960196821F4E02141F480311960116824
:1004F00021F0E04141F080511160016821F4401188
:1005000041F400110160116821F4403111601A6852
:1005100022F040521A6002B070471A6891033FF50A
:100520005DAF019A013A54E70044025848BE2100E9
:10053000184402581C440258284402581220200033
:10054000770203072F0201018808BF000C480258F8
:100550001848025804480258F44402582C04005821
:100560000020005210440258544402585844025883
:100570005044025808B5204B012100201A6842F06F
:1005800001021A601D4A11601D4A10601D4A196857
:100590000A401D4942F010021A601C4A11601A6894
:1005A00022F480221A60186600F07AF8FFF708FF3C
:1005B000174A136843F0006343F001031360154BBF
:1005C0001A681A6053F8082C43F8082C124A13686A
:1005D00043F0805343F09F031360104B1A681A6076
:1005E0005A685A609A689A6053F8042C43F8042CAD
:1005F000DA68DA6008BD00BF004402580881005183
:100600001044025867EFFEEA0000FF012C44025834
:10061000D8440258DC440258E0440258E8440258E6
:100620007047FFEC30B4EFF3118400238022EFF326
:10063000108372B682F3118883F31088BFF34F8F53
:10064000154B164A1B68118803F4807578B1013187
:100650001180B5B112886AB10023BFF34F8FE4B2A5
:1006600084F31188B3B1042030BC00F05CB831B120
:100670000139EDE723F48073074A1360ECE7002D9E
:10068000F8D11288002AE7D043F48073024A13603D
:100690000123E2E730BC704700480258E002002422
:1006A000EFF3118200238021EFF3108372B681F300
:1006B000118883F3108806490B6823F480730B605C
:1006C0000021044B1980D3B283F31188FFF7AABF2E
:1006D00000480258E0020024F8B5074C07460D46D2
:1006E0002668216000F03DF93846294600F0B6FB47
:1006F00020682660F8BD00BFE402002430B5EFF3A7
:10070000118400238025EFF3108372B685F31188DE
:1007100083F31088036823EA0101E3B20A4302600D
:1007200083F3118830BD82B0002245F26161B0F5DB
:100730007A7F0BD8002240F6A201642811D800224B
:100740000A2818D8002200BB02B070470192019B12
:100750008B4202DDA0F57A70E9E7019B013301933A
:10076000F5E70192019B8B4201DD6438E5E7019BCF
:1007700001330193F6E70192019BDC2B01DD0A387E
:10078000DEE7019B01330193F6E70192019B152BF4
:1007900001DD0138D7E7019B01330193F6E7FFEC58
:1007A000BFF34F8FBFF36F8F064B00221A60064ACC
:1007B000136843F400331360BFF34F8FBFF36F8FA1
:1007C000704700BF50EF00E014ED00E00F2810B5B7
:1007D00031DDA0F110041F2C0ADC03F1604303F5A6
:1007E00061430B60012303FA04F4146000201CE051
:1007F0003F2C08D81C4C30381C440C60012303FAF1
:1008000000F01060F2E75F2C04D8184C50381C44FC
:100810000C60F3E77F2C04D8154C70381C440C6036
:10082000ECE7952C02D94FF0FF3010BD114C9038F9
:100830001C440C60E2E7104B04280B6003D14FF41A
:1008400080331360D2E7052802D14FF40033F8E774
:10085000062802D14FF48023F3E70F28E3D1074B9A
:100860000B600123EDE700BF04E100E008E100E0D8
:100870000CE100E010E100E024ED00E010E000E019
:1008800038B51B4B4FF0FF311A4A1C6804F00F04B7
:1008900001342346013B42F8041BFBD1164AE40015
:1008A000164B174D1A604FF08033164A1360A2F6AC
:1008B00018122B60C2F82039013C42F8043BFBD1EE
:1008C000114B224611490B201C6000F09FFA224672
:1008D0000F49032000F09AFA2B6823F07F4343F07E
:1008E000E0432B60F02383F3118862B638BD00BF6C
:1008F00004E000E080E100E00000000808ED00E016
:100900001CED00E018ED00E0E40200248909000875
:100910006509000813B5802301AA69460446FFF75C
:1009200055FF20B90F2CDDE9003102DD196002B05E
:1009300010BD1A6822EA01021A60F8E713B5002315
:1009400001AA69460446FFF741FF20B90F2CDDE9F3
:10095000003102DD196002B010BD1A680A431A6046
:10096000F9E7704708B5EFF3118300238022EFF316
:10097000108372B682F3118883F3108887210148AF
:1009800000F036F9689A0008CB6E012B10B50C46C2
:1009900009D003D3022B0AD0002010BDD422086F47
:1009A00000F01EF8F8E70A6F044B1A60F4E7D4224F
:1009B000086F00F015F8626FF6E700BFE40200244C
:1009C00018DF88DFCD06CD767CD30CD3D982D9123F
:1009D0002C00050A0F14191E232800BFAFF3008056
:1009E00000B501B400F004F801BC00BDAFF3008015
:1009F00000B5042A60DB00F0030E61F3830E7A4B2E
:100A0000D3E80EF0AFF30080AFF30080AFF30080C7
:100A100011F8013B00F8013BA2F1010211F8013B82
:100A200000F8013BA2F1010211F8013B00F8013B83
:100A3000A2F101022DE9F01F282A07DBB1E8F81F17
:100A4000A0E8F81FA2F12802282AF7DADFF89CE1D3
:100A50004FEA920BDEE80BF051F8043B40F8043B00
:100A600026E0B1E81800A0E8180021E0B1E838005D
:100A7000A0E838001CE0B1E87800A0E8780017E0B2
:100A8000B1E8F800A0E8F80012E0B1E8F801A0E849
:100A9000F8010DE0B1E8F803A0E8F80308E0B1E8D8
:100AA000F807A0E8F80703E0B1E8F80FA0E8F80FAE
:100AB000BDE8F01F02F00302002A08BF00BD11F8D4
:100AC000013B00F8013B013A08BF00BD11F8013BB2
:100AD00000F8013B013A08BF00BD11F8013B00F8E6
:100AE000013B00BDAFF30080AFF30080AFF30080A7
:100AF00011F8013B00F8013BA2F1010211F8013BA2
:100B000000F8013BA2F1010211F8013B00F8013BA2
:100B1000A2F10102282A35DB2DE9F01FB1E8F81F08
:100B200020F8023B4FEA134364F31F434FEA144497
:100B300065F31F444FEA154566F31F454FEA164615
:100B400067F31F464FEA174768F31F474FEA1848F5
:100B500069F31F484FEA19496AF31F494FEA1A4AD5
:100B60006BF31F4A4FEA1B4B6CF31F4BA0E8F80FC7
:100B70004FEA1C4C20F802CBA2F12802282ACDDA39
:100B8000BDE8F01F042A97DB51F8043B20F8023B34
:100B90004FEA134320F8023BA2F10402BAE711F82E
:100BA000013B00F8013BA2F1010211F8013B00F802
:100BB000013BA2F1010211F8013B00F8013BA2F157
:100BC0000102042AFFF678AF51F8043B00F8013B1C
:100BD0004FEA132320F8023B4FEA134300F8013B8E
:100BE000A2F10402EDE70000C0090008D0090008E6
:100BF00008B501F0ADFB012000F09EFB08B5012017
:100C000000F09AFB704700F009B8002070470021FF
:100C1000084601F049BA04F0C9BDFFEC014801F0F3
:100C200093BA00BF080C02007047FFEC514E01233D
:100C30000024514D33704FF4B472504B05F5A47835
:100C400083B54F4F214628463C607C601C605C6049
:100C50004C4B1C605C604C4B1C605C604B4B1C60E4
:100C60005C604B4B1C605C6003F0C0FE03231822E9
:100C700048494046AB76484BC5E904330623AB836D
:100C800003F00CFF454B39462846C5F86431C3E9EB
:100C9000008403F069FD424B01A968461D600223F0
:100CA000404C337001F030FADDE9000103F062FAE4
:100CB000042323602368012B50DD2068C00003F06B
:100CC0006FFA0022384B4FF6FF7C174618602068F9
:100CD0001968904245DC226800240D601B68264894
:100CE0009C80297F00F046FB234801F0F3FB18218C
:100CF000214801F0C1FCAB689B6803601E4800F00E
:100D000053FBAB6801221A71284B1C8003233370FC
:100D100006F0BCFD264B0BB100F07EFB254B0BB162
:100D200001F096F9244B0BB107F086FA234B0BB177
:100D300000F0C2FF01F0AEFB04230F48337000F057
:100D400055FB05F0BFFD00F0B9F80523337000F046
:100D50004BF800F0C1F801F0E2FCFCE723685B000F
:100D6000A7E741F83270196801EBC2010132A1F81E
:100D700004C0ACE768040024F00200246C040024E2
:100D8000780400248C0400249404002484040024A7
:100D900058040024809A00082D0C0008E802002462
:100DA00080040024640400247404002460040024EB
:100DB000191400085120000839820008B91C0008E5
:100DC00013B50024FFF723FF054B4FF4386200945E
:100DD0006421044800F0D9F8204602B010BD00BFDD
:100DE000DD930008D79A000813B50024054B4FF493
:100DF0000062FE210094044800F0E0F8204602B0B2
:100E000010BD00BFC10D0008CC9A0008A52870B520
:100E100006460C461AD8EFF3118500238021EFF324
:100E2000108372B681F3118883F310881CB9FFF721
:100E300071FD2246074C0848EDB240F8364000EB01
:100E4000C600426085F31188002070BD6FF0150068
:100E5000FBE700BF990E00089C040024A52808B5F4
:100E60000CD8094A52F830305BB102EBC00252682C
:100E70009847064B1A68064B1A6008BD0022054BBE
:100E8000F6E71A46FBE700BF9C0400247804002420
:100E900080040024990E000808B5EFF311830023A5
:100EA0008022EFF3108372B682F3118883F31088E7
:100EB00033210148FFF79CFEDC9A0008054B10B572
:100EC0001C682CB101F038FB10B9E38B0133E383CC
:100ED000002010BD7804002438B5144B1C6814B3EE
:100EE00001F02AFBF8B9EFF3118500238022EFF31C
:100EF000108372B682F3118883F31088B4F91E3020
:100F0000002BC4BF03F1FF33E383B4F91E30002B81
:100F100006DC0023E383064B1B680BB101F014FBD6
:100F2000EDB285F31188002038BD00BF780400249D
:100F30006C0400242DE9FF4104464FF4B470884648
:100F400016461F4603F03CF90546D8B10C9B2146D6
:100F5000A0F81C80324602930B9B01930A9B0093DE
:100F60003B4600F035F8041E06DA284603F010F977
:100F7000204604B0BDE8F0812846B5F90C4000F0E9
:100F8000A5F9F5E76FF00B04F2E71FB5069C009298
:100F90000A46CDE9013400231946FFF7CBFF04B020
:100FA00010BD1FB5079C0294069CCDE90034134682
:100FB0000A460221FFF7BEFF04B010BD13B5049C22
:100FC000CDE9003413460022FFF7EBFF02B010BD5D
:100FD0002DE9F347067F89460446924631461F466F
:100FE000DDF8288000F0C6F9051E44DB204606F037
:100FF000030600F006FA051E38DB77B14246394693
:10100000204601F075FB051E32DB1821204601F059
:1010100033FB88B96FF00B0528E0324608F1180160
:10102000204601F0FDF9051EEFDAA36B03B331464C
:10103000204601F0A5FA1BE0A3685146104A9B68C0
:101040000360204600960B9B00F01EF8051E0DDB8A
:101050000C9A4946204600F0CFF8204600F0A4F94B
:10106000054640B10749204603F08AFB002FDCD03B
:10107000204600F0A1F9284602B0BDE8F08700BF85
:10108000F1120008580400242DE9F04F85B0044601
:10109000CDE900120293EFF3118600238022EFF3D3
:1010A000108372B682F3118883F31088DFF84081D1
:1010B000DFF84091C246B8F8003000204A4F0133B3
:1010C000D9F800B039461BB23D68A8420EDB38683B
:1010D0000391000103F064F80399054600284FD1FD
:1010E000F6B286F311886FF00B0042E0012B3D68E9
:1010F000B8BF0123013D1D404FEAC50C5BF83550D8
:101100000BEB0C0E002D37D1CEF80040F6B2D9F81B
:101110000020AAF800309444ACF80430A38186F390
:1011200011889DF800302946032023766376019BC1
:101130002361029B6361A38B23F003029DF8383087
:1011400003F00303134304F1440223F0C003A38319
:1011500000F0C2F92046A57601F0BCF9FFF7AEFE1B
:101160002249204603F000FB0423A376FFF7B4FED8
:10117000284605B0BDE8F08F013301301BB2A3E76C
:101180003B684FF6FF7C5B003B6000231F4608680E
:1011900083420FDB584600274FF0020C0B680830E3
:1011A00093FBFCF39F420DDB584602F0F1FFC9F8B8
:1011B000005080E705EBC30045F833700133A0F819
:1011C00004C0E4E70B68013730F904EC013B50F848
:1011D000082C0EEA030305EBC30E45F8332030F963
:1011E000043CAEF80430D9E7640400245804002419
:1011F0006004002474040024334B2DE9F74F0029C8
:1012000014BF8946994605460024174649461822C8
:1012100000F5A47003F042FC85F86041484603F0F5
:1012200035FC461C2FBB3C4602342846A400A119BD
:1012300001F022FA8246002842D000EB0408083C64
:10124000043FC0F80080484603F020FC06464946AB
:1012500054440136D1464046464403F00FFC4C4509
:101260001AD1002048F8040CC5F864A103B0BDE809
:10127000F08F40F2011857F824000028D4D003F072
:1012800005FC01306B6B06449E4216D20134444586
:10129000F1D16FF00600E9E749F8046F57F8041F31
:1012A0000846019103F0F2FB8346019930460BF1A9
:1012B000010B03F0E3FB5E44D1E76FF05A00D5E782
:1012C0006FF00B00D2E700BFF49A000810B5EFF3FF
:1012D000118400238022EFF3108372B682F3118809
:1012E00083F3108801F0E4F9E4B284F3118810BDAF
:1012F00038B5104B1C68204600F0CAFBD4F86421B6
:10130000012040F2011152F820304BB9A38B6569DE
:1013100003F00303022B08D11146A84700F00CF894
:1013200001308842EFD10120F8E70146284603F05A
:1013300035FAF8E77804002408B5054BC4B200225A
:101340001B682146184600F0C9FB204601F08CF8C6
:101350007804002410B5044658B1806820B100F02C
:10136000A3F8A06802F014FF2046BDE8104002F088
:101370000FBF10BD38B505464FF4867002F020FF50
:10138000044670B1342002F01BFFA06030B101228E
:10139000002103F02DFA0020AC6038BD2046FFF795
:1013A000D9FF6FF00B00F8E7B0F90C20836800203C
:1013B0001A8001225A71704738B58468054634B1E5
:1013C0006379012B04D9013B63710023AB6038BD05
:1013D000204600F065F904F1200006F086FA204668
:1013E00003F026F92046FFF7B5FFEEE710B50446F7
:1013F0008068203006F075FA2046BDE8104000F005
:10140000B0BB10B504468068203006F06AFA20466A
:10141000BDE8104000F0A5BB0023074A10B41846F1
:10142000064C9C50D11808334860B3F5A66FF8D12C
:101430005DF8044BFFF724BA9C040024990E0008C1
:1014400070B5044650B3B0F90C00E0B1EFF311826F
:1014500000238025EFF3108372B685F3118883F3A0
:1014600010880F4B00261B68013B03400D480568A0
:1014700045F83360006800EBC3034FF6FF709880B7
:10148000D3B283F31188A36B13B1204601F078F82F
:101490002046FFF791FF204602F07AFE002070BD43
:1014A000640400247404002430B103881B0401D4B4
:1014B00001230380002070476FF01500704710B5BE
:1014C000FFF7F2FF041E05DA644203F08CF80460B3
:1014D0004FF0FF34204610BDF8B51746194B0646AD
:1014E0000C461D68FFF7EAFC0FB16B6C3B60D4B192
:1014F000EFF3118300228021EFF3108272B681F3A3
:10150000118882F31088022E11D0032E14D0012EE0
:1015100014D16A6C21680A4300246A64DBB283F345
:10152000118800F011F8FFF7D7FC2046F8BD2168BC
:101530006A6C22EA0102EFE72268EDE76FF015041A
:10154000ECE700BF78040024174B37B51D68FFF7A0
:10155000B5FC6C6C284600F09DFCE443044001940B
:1015600024B9FFF7B9FC204603B030BD01A800F054
:101570006FF8431C044610D0014601A803F060F93F
:101580002146284600F012F8044630B1011D2846D5
:1015900000F09AF8204600F02DF8019B002BE5D1D1
:1015A000FFF79AFC0120DFE77804002438B5836850
:1015B000EFF3118500228020EFF3108272B680F3E2
:1015C000118882F3108800205C6974B122798A4204
:1015D00006D103F1140130B9084603F09FF804E086
:1015E00020462468F1E703F0A3F8EDB285F31188F3
:1015F000204638BD10B5037B83B9EFF311848022F8
:10160000EFF3108372B682F3118883F310880E49CA
:1016100003F064F8E4B284F3118810BD022B0CD1FE
:10162000EFF3118400238022EFF3108372B682F36C
:10163000118883F310880549EAE7012BEDD1BDE855
:10164000104002F0A5BD00BFEC090024E40900240D
:1016500038B5054601242146284603F002F920B991
:101660000134202CF7D14FF0FF34204638BD38B577
:10167000044600F14C05284603F050F850B904F137
:101680005405284603F04AF838B94FF0FF32C4E950
:10169000112038BD00F058FCEDE700F055FCF0E7F4
:1016A00038B5044600F10C05284603F037F828B990
:1016B0001434204603F032F818B938BD00F06EFB40
:1016C000F2E7FFF797FFF4E72DE9F0410E460978BE
:1016D000044629B3443003F0C4F8012807467ED1FC
:1016E000EFF3118500238022EFF3108372B682F3AB
:1016F000118883F31088A37EEDB2062B12D13178C6
:1017000004F1480003F0ADF860B133682046E365AA
:10171000736823660023A36400F0CAFF85F3118871
:101720000025C0E085F31188A7683178EFF31183B5
:1017300000228020EFF3108272B680F3118882F3CA
:1017400010887C6914B122798A4208D1DBB283F314
:10175000118834B1336863607368A360E0E724687C
:10176000F0E700F0E9FEF8B1544802F0D7FF20B9E5
:10177000534802F0D3FF0028D2D033684360736827
:101780008360EFF3118400238022EFF3108372B69D
:1017900082F3118883F3108807F11401E4B202F098
:1017A0009DFF84F31188BBE7EFF3118500238022AE
:1017B000EFF3108372B682F3118883F310883F48E9
:1017C000EDB202F0ABFF85F311880028D5D11020CF
:1017D00002F0E6FC0028A3D001230373CDE7FFF756
:1017E0006DFB3178A06800F073FB054640B3436899
:1017F0002BB300F07FFB002858D06B684360AA68C9
:101800008260EB689B0604D4317801238B4013433C
:1018100083603368C36073680361EFF3118500234D
:101820008022EFF3108372B682F3118883F310885D
:1018300004F14C01EDB202F051FF85F3118800254F
:10184000FFF74AFBEFF3118800238022EFF31083A8
:1018500072B682F3118883F310881A49204600F08B
:10186000A1FEA37E062B08D133682046E36573688A
:1018700023660023A36400F01BFF5FFA88F888F357
:101880001188002F15D1A37E052B03D104212046FA
:1018900000F0F4F9A37E072B05D13378082B02D191
:1018A000204600F0C0F92846BDE8F0816FF00B0536
:1018B000C6E7F8DA6FF01505F5E700BFEC0900247C
:1018C000E4090024E318000810B50C4600F062F9A2
:1018D00020B12146BDE81040FFF7F6BE6FF00200D0
:1018E00010BD2DE9F04F00F14C0385B004464FF0D8
:1018F000800900F154080393EFF31183019AEFF389
:10190000108272B689F3118882F31088A78B5FFA70
:1019100083FA019217F4007704D08AF3118805B096
:10192000BDE8F08F039802F0F9FE06460028F4D0D7
:10193000A28B414642F40072A28302F0CFFED4F89B
:1019400044B0B5684BEA050565648AF3118873688D
:101950003A4606F10C01307B9847EFF31187029B62
:10196000EFF3108372B689F3118883F31088029322
:101970004146A38B3046FFB223F40073A383636C0C
:101980005D4083EA0B031D4085EA0B05656402F0A8
:10199000AFFE87F31188FFF7D7FD304600F0D4FA89
:1019A000AAE77047054B10B51C68FFF787FA204679
:1019B00000F018F9BDE81040FFF78EBA7804002453
:1019C00008B5044B186800F0AEF810B90120FFF715
:1019D000B3FC08BD7804002408B580681C3002F010
:1019E00040FF0028D4BF0020012008BD0023094A81
:1019F00010B512F83340D900844205D10A4450781A
:101A0000C04300F0010010BD01330B2BF1D10120C8
:101A1000F9E700BF009B000838B585685AB100237C
:101A20001A4A12F83340D800A14218D1024405F1F5
:101A30001C005468BCB9EFF3118400238022EFF33B
:101A4000108372B682F3118883F3108805F11C00AD
:101A5000E4B202F0F5FE84F31188002413E00133B0
:101A60000B2BDED1E7E7EFF3118500238022EFF3A4
:101A7000108372B682F3118883F3108802F0D3FECC
:101A8000EDB285F31188204638BD00BF009B0008E9
:101A90002DE9FF41856800240F4F1C35A0462846DC
:101AA00002F0DBFE3B195B6873B1E65D01A9002221
:101AB0003046CDE9013802230393012300F074F985
:101AC0003146284602F0AFFE0834582CEAD10020F7
:101AD00004B0BDE8F08100BF009B000810B5838B07
:101AE00004461B0515D43AB9806828B14379012B07
:101AF00002D1283002F0D0FE204600F00BF820463C
:101B0000FFF75AFC2046FFF7B2FDA38B43F40063B6
:101B1000A38310BD10B5044600F020F82046BDE8B0
:101B2000104000F092B8EFF3118100238022EFF310
:101B3000108372B682F3118883F31088838BC9B245
:101B400013F0040206D043F01003838381F311885D
:101B50000120704781F3118810467047243000F04F
:101B600021BA10B50446806802F042FD00232246E7
:101B70000121184606F049FA2246002306210120D9
:101B800006F043FA002322460621022006F03DFA21
:101B9000002010BD002810B51DDBEFF311820023DB
:101BA0008021EFF3108372B681F3118883F31088DC
:101BB0000A4B0B491B680968013B034001EBC30456
:101BC000B4F9044084420CBF51F833000020D3B272
:101BD00083F3118810BD0020FCE700BF64040024DB
:101BE0007404002438B50546EFF3118400238022E5
:101BF000EFF3108372B682F3118883F31088837E2B
:101C0000043B032B0BD800F015FA042307212846C8
:101C10002B8400F0FBF9E4B284F3118838BD07216E
:101C200000F0C4FBF7E710B5EFF311840023802226
:101C3000EFF3108372B682F3118883F3108800F0FB
:101C400037FDE4B284F3118810BDEFF31182002355
:101C50008021EFF3108372B681F3118883F310882B
:101C6000837E052B06D1016C0B8801331BB20B80E0
:101C700000230364D3B283F31188704738B5EFF3C0
:101C8000118400238025EFF3108372B685F3118849
:101C900083F31088837E052B09D1056C2B880133D3
:101CA0001BB22B8000230184036400F001FDE4B229
:101CB00084F3118838BDFFECF8B50024284B294D7A
:101CC0006020C3E90044284BC3E90044274BC3E923
:101CD0000044274BC5E90044C3E9004402F060FA20
:101CE00050B100F1600600F118070475294602F0B2
:101CF000F5FCBE423846F6D1C02002F051FA60B180
:101D000000F1C0040227184E00F11805077531468E
:101D100002F0E4FCAC422846F6D1402002F040FA42
:101D200060B100F140040027104E00F11005077368
:101D3000314602F0D3FCAC422846F6D1802002F0B6
:101D40002FFA60B100F180040227094E00F110055E
:101D50000773314602F0C2FCA5422846F6D1F8BD11
:101D6000CC090024D4090024DC090024EC09002457
:101D7000E409002470B5502002F012FA50B100F1CD
:101D80005004054E00F11405314602F0A7FCAC42A8
:101D90002846F7D170BD00BFCC090024014902F0EC
:101DA0009DBC00BFCC0900242DE9F8431546374AF5
:101DB0001F280746D2F800800E46D8F8089003D9AD
:101DC0006FF01500BDE8F88341B93946484600F088
:101DD0007FF8044665B916BB0020F3E7002BF4D169
:101DE0000B68012BF1D0FFF701FE0028EDD1E7E7EA
:101DF00039464046FFF7F0FD30B100230122C5E926
:101E000000230223AB60E6E72CB163682B60A36874
:101E10006B60E368F6E7C5E90044AC60DBE7356872
:101E2000012D11D12A4639464046FFF7F5FD0546FA
:101E300085B9002CD0D0204609F10C0102F058FCE5
:101E40002046FFF7ABFFC7E7002239464046FFF7C1
:101E5000E3FDEDE78CB90E4802F060FC044630B9B2
:101E6000FFF788FF0A4802F059FC044658B127746E
:101E700009F10C01204602F031FC65607368A36033
:101E8000B368E360A8E76FF00B009BE778040024D9
:101E9000CC09002473B5002302AE826846F8043DE5
:101EA000EFF311858021EFF3108372B681F311886F
:101EB00083F3108854692CB9EDB285F31188019829
:101EC00002B070BD2179304602F0ADFC2468F2E723
:101ED00038B50D46044640B1FEF7F0FFE46814B192
:101EE000237CAB4203D1FEF7F7FF204638BD2468C0
:101EF000F5E7FFEC10B500F01FFB40B1104802F011
:101F00000DFCE0B90F48BDE8104002F007BCEFF34C
:101F1000118400238022EFF3108372B682F31188BC
:101F200083F310880648E4B202F0F8FB84F31188CA
:101F300028B9182002F034F908B10123037510BD47
:101F4000D4090024DC09002410B5037D83B9EFF324
:101F500011848022EFF3108372B682F3118883F329
:101F600010880E4902F0BAFBE4B284F3118810BD68
:101F7000022B0CD1EFF3118400238022EFF31083A6
:101F800072B682F3118883F310880549EAE7012BC2
:101F9000EDD1BDE8104002F0FBB800BFD409002429
:101FA000DC09002438B5EFF3118500238022EFF31C
:101FB000108372B682F3118883F31088F8B14368F6
:101FC000EBB1114B00221C68E4B1844223680FD1AD
:101FD0001BB19968A0680144996062B10A49104632
:101FE00002F0A6FB00206060EDB285F3118838BDD9
:101FF00022461C46E8E7044802F090FBF2E76FF047
:102000001500F1E72368FFDEF409002438B50C461B
:10201000074B054653F8311003EBC4031B79DB076C
:1020200003D500F01DF8AC7638BD02F091FBFAE75D
:102030008C9A0008054B827E10B553F83210044686
:1020400002F09EFB0023A37610BD00BF8C9A00080F
:10205000024B0022C3E90022704700BFF4090024AC
:1020600010B50B68027EB3B11C7E944206D25A684A
:1020700062B9C0E900325860086013E01B68F2E7FB
:10208000C0E900321060486000200CE0C0E9003276
:1020900010605860F8E74A68002AF1D1C0E90033BF
:1020A000C1E90000012010BD37B5124D2C682CB1DC
:1020B000114802F0DFFB012003B030BD0F4802F0F1
:1020C000D9FB40F2011369464FF60C70ADF80030B1
:1020D0008DF80240019503F077FE011E04DA4942B3
:1020E000074802F0C7FBE6E7064802F0C3FB2046BC
:1020F000E2E700BFFC090024589B00087B9B000816
:10210000A69B0008E59B0008044B1B680360C3F115
:10211000105303F500230B60704700BF649A00085A
:10212000C0F30313072B0AD8064A52F8232032B112
:1021300000F00F00012319B103FA00F0906170471D
:102140001030F9E7209C00082DE9F843C0F303178D
:102150000446072F00F2DB806E4B53F82760002EF9
:1021600000F0D58000F4402300F00F05B3F5002FF8
:1021700000F0B980B3F5402F00F0B380B3F5802FA5
:1021800000F0A9800020EFF3118100238022EFF3FB
:10219000108372B682F3118883F31088022840F00E
:1021A000A480C4F3033EBEF1000F14D0072D4FF0FE
:1021B0000F088BBFA5F108032B46242220229B0089
:1021C00052F806C008FA03F80EFA03F32CEA080CDA
:1021D00043EA0C0393514FEA45080322336803286E
:1021E00002FA08F26FEA020202EA030C00FA08F3AC
:1021F00043EA0C0333607BD004F44033B3F5803FF3
:1022000079D0B3F5003F0CBF4FF0020C4FF0000C3B
:10221000F3680CFA08FC13404CEA0303F360BEF1C8
:10222000000F13D1072D4FF00F098BBFA5F1080345
:102230002B464FF0240C4FF0200C9B005CF806E07E
:1022400009FA03F32EEA03034CF8063000F1FF3CD1
:10225000BCF1010F56D804F44063B3F5006F4DD0C4
:10226000B3F5406F4CD0A3F5806EDEF1000343EB75
:102270000E03D6F808E003FA08F3BCF1010F02EAF6
:102280000E0243EA02034FF00102B36002FA05F2C4
:10229000736839D814F4007F36D013430128736073
:1022A00013D0E30511D504F00C04AD000F2204F1A6
:1022B000B04405F00C05D4F80834AA4007FA05F537
:1022C00023EA02031D43C4F80854C9B281F31188FC
:1022D0000020BDE8F883C0F30021FFF721FF0120B3
:1022E00051E703204FE702204DE74FF0000E72E761
:1022F0004FF0000C8CE74FF0010C89E70223B8E7A0
:102300000323B6E70023B4E723EA0203C6E76FF02E
:102310001500DEE7209C0008C0B2FFF715BFFFECF8
:10232000C0F30313072B0ED8084A52F8233053B1D9
:102330001A6900F00F00012303FA00F0104214BFE5
:102340001846002070470020704700BF209C0008FE
:1023500008B504F0ABFA04F0A9FA04F0A7FA104BA0
:102360001B6873B1EFF3118300238022EFF3108316
:1023700072B682F3118883F31088002007F004F905
:10238000FBE700F0D9F848B1064B1B681B68002B2F
:10239000E8D00020BDE8084007F0F6B8024BF4E7AB
:1023A000E402002480040024780400242DE9F04194
:1023B00007468846114C266805F074FF41460546DD
:1023C0003846FFF723FE0E4B1B681BB105F07EFF5E
:1023D0000543EDB24DB10B4D06F17400296831B1E2
:1023E00000F012F8236874332B60BDE8F081216897
:1023F000BDE8F041743100F0AEB900BF78040024AC
:102400006C040024E4020024814208D0043801F165
:10241000D40351F8042B8B4240F8042FF9D17047B4
:1024200038B50731836B044621F007052BB1436BA8
:10243000AB4202D0114600F0A3F8A36B23B92946A2
:10244000082001F0B5FEA063A06B50B1E0632946FF
:10245000656300F065F9A38B002043F48053A383E8
:1024600038BD4FF0FF30FBE7094C08B52368EFF3A8
:10247000118300238022EFF3108372B682F3118858
:1024800083F3108806F0A8F82068743000F05EF935
:102490007804002408B50B4A00230B4913600B4A4B
:1024A00042F823100133802BFAD1094B0BB1AFF363
:1024B000008005F0C5F900F083FBBDE8084001F09D
:1024C000E7BC00BFE4020024EFBEADDEE000002464
:1024D0000000000038B5B0F90C10044600F16405A6
:1024E00051B9144B186840F2EE23A0F2EE2063635A
:1024F000C4E90E0000F014F9E4220021284602F09D
:1025000075FAE36B626B13446367236923F001037D
:10251000C4F8F8304FF08073C4F8FC306FF0160345
:10252000C4F89C300023C4F84031C4F84431F0238F
:10253000A36738BD649A0008024B1868003018BFC2
:1025400001207047E402002470B50B4D2C6805F0A3
:10255000BDFE48B1094E04F17400316829B1FFF79E
:1025600053FF2B687433336070BD2968BDE8704039
:10257000743100F0F0B800BF78040024E4020024B5
:1025800010B50446806B20B1A38BDB0401D501F0AC
:10259000FFFDA38B23F48053A3830023C4E90E33F0
:1025A000636310BD426E002A30D1194A126882421C
:1025B0001AD1184B1B6803B90847516602F1740021
:1025C000D3F8841091665968D166D3F888101167E2
:1025D0001149C3F88410802159604FF08071C3F80D
:1025E00088101946FFF710BFD0F8F82041668266C0
:1025F000826FC266D0F8FC200267074AC0F8F82054
:10260000802282674FF08072C0F8FC20704700BFC4
:1026100078040024E40200241D260008154B30B580
:102620001C68B7B001F0DFFF056804F1740101A870
:10263000FFF7EAFEF02383F3118862B6636E20464B
:102640009847EFF3118300238022EFF3108372B6D3
:1026500082F3118883F3108801F0C5FF0560A36E33
:1026600001A82293E36E0293236F239300236366F2
:1026700000F06CF87804002438B50731836B044609
:1026800021F007057BB1436BAB420ED9C36B2A46E1
:102690000021184602F0AAF9E26B616B03462A4456
:1026A000491BE2636163184638BD0023FBE7FFEC7A
:1026B00070B506460C4D2C68FFF7BCFC304605F0A3
:1026C000CDFD48B1094E04F17400316829B1FFF71E
:1026D0009BFE2B687433336070BD2968BDE8704081
:1026E000743100F038B800BF78040024E4020024FC
:1026F00070B5836B06460D46144623B1017F01F089
:102700000301FFF73DFF2919284621F00701491B66
:10271000C6E90E55716300F003F8002070BD7047E4
:10272000C31C23F0030351B1084420F00300C01A76
:10273000054A20F003001844834202D170476846DE
:10274000F5E71A600433F7E7EFBEADDE01464FF060
:10275000010000DF70470A4601464FF0020000DF2B
:10276000704710B5846E01F4D873A0F8501001F0D2
:102770000101226822F4D87213432360826E9368A9
:1027800023F001031943916010BD10B5EFF31184DC
:1027900000238022EFF3108372B682F3118883F353
:1027A0001088FFF7DEFFE4B284F3118810BDFFEC60
:1027B000F0B5C36BEFF3118400228021EFF3108298
:1027C00072B681F3118882F31088996E0A6822F03C
:1027D000010002F001050860DE6D5F6E710801EB1B
:1027E0004701B1FBF6F164293AD9013122F40040E6
:1027F000490820F001009A6E10609A6ED16093F83B
:102800005610234A012902EA000233D142F4C06281
:1028100093F85700092802D0082830D179B342F440
:102820008052996E0A60986E93F85860416821F45E
:1028300040510EB141F400514160986E93F85960D7
:10284000816821F440711EB15E6F0EB141F4807158
:1028500081602A439B6EE4B21A6084F31188F0BD54
:10286000C1F3420221F00F0140F400400904090CB9
:102870001143C0E7022908BF42F48062C8E7B3F8F9
:102880005610B1F5E06F08BF42F08052C9E700BFB3
:10289000FEE9FFEFC36B9A6E506AB3F8522040EA2C
:1028A0000242C0B20A600022A3F85220704710B55D
:1028B000C06BEFF3118400238022EFF3108372B614
:1028C00082F3118883F31088B0F8503039B143F0A7
:1028D0002001FFF75AFFE4B284F3118810BD23F4FE
:1028E000907121F00101F4E7C36B9B6ED869C0F3CE
:1028F00040107047C36B9B6E99627047C36B9B6EB1
:10290000D869C0F3C010704738B50546C06BEFF307
:10291000118400238022EFF3108372B682F31188B2
:1029200083F31088B0F8503051B143EA0201FFF749
:102930002CFF284603F024FFE4B284F3118838BD4D
:1029400023F08001FFF721FFF6E738B583685D6962
:1029500040F201139942EC6B05D0B1F5817F29D08B
:102960006FF0180023E0002A4CD094F85630FBB1E9
:10297000012B4FF480710CBF4FF4007300230B4305
:1029800094F858101046002914BF402100210B4331
:1029900094F85910002943F0300314BF4FF0004160
:1029A00000210B439360E16D02F08AF8002038BDEE
:1029B0001946E4E732B3936803F03001302921D19E
:1029C000002B01DA616FE9B113F4807117D013F4B1
:1029D000007F14BF0123022384F856309368104609
:1029E000C3F3801384F858309368DB0F84F85930B0
:1029F00002F086F8E0652846FFF7DAFED6E784F8AD
:102A00005610EBE76FF01500D1E710B5C46B94F8E2
:102A10006000FDF77FFF002294F860001146BDE8DA
:102A20001040FEF7F3B9FFEC38B5C46B06492246F7
:102A300094F86000FEF7EAF9054618B994F86000CA
:102A4000FDF77CFF284638BD6D2A000810B5C36B22
:102A5000144693F859302BB1836B9B6922B1002146
:102A600098472346184610BD0121F9E710B51446D2
:102A7000926ED3699BB29806A4F8523013D5B4F87D
:102A8000501089060FD5204603F0B1FEB4F852303D
:102A90001A0606D5B4F850301B0602D5204603F0BE
:102AA0006FFE002010BD13F00E0FEFD00E23136247
:102AB000ECE7FFEC38B5C46B00210546A36E196046
:102AC000C36B9A6E1E4B9A4204D14FF480221D486C
:102AD000FDF714FEE06EFFF737FB206FFFF734FBC6
:102AE000606F08B1FFF730FBA26E94F8581053687E
:102AF00023F47D5309B143F4005353602846A26E7A
:102B0000114B11680B401360A26E94F85510936836
:102B100023F4E06323F0010343EA41639360FFF78A
:102B200047FEA26E0020136843F0005343F00D03EC
:102B300013600123A4F8500084F8543038BD00BF5E
:102B400000480040E844025803BEFF33F8B50025B2
:102B5000C46B074684F85450EFF3118680222B464D
:102B6000EFF3108372B682F3118883F3108829463D
:102B70002046FFF7F6FDF6B286F31188FB6B9A6EDE
:102B80000D4B9A4205D12A464FF480210B48FDF7A0
:102B9000B5FDA26E136823F00D031360E06EFFF71E
:102BA000BBFB206FFFF7B8FB606F18B1BDE8F840C2
:102BB000FFF7B2BBF8BD00BF00480040E844025830
:102BC0007FB50B49684601F059FF0023094D1C46AB
:102BD00055F8241039B15E1C303368468DF8093041
:102BE00003F006FC33460134082CF1D104B070BD6B
:102BF000409C00084C9C0008704738B503690446A7
:102C00002BB15A69026102B9426100225A61627EA7
:102C1000207EC2F3C00520B9E068007C60F3C302E7
:102C2000627659812046DA6819469047637E65F3DB
:102C3000C303637638BD37B50446C0680A4680B121
:102C40000368B4F85E10009121469D6804F11D03ED
:102C5000A847002803DA237C43F00103237403B060
:102C600030BD6FF00400F6E7F0B5047E3CB31346C8
:102C70006401144FE5592E0416D4AE0343F080537B
:102C8000114E48BF45F0806543F400432E4043EAAF
:102C900081433343E351437EC28061F3010303F078
:102CA000F3036FF386134376037E0020074903F195
:102CB000100201230C68934023430B60F0BD2146B2
:102CC0002346D5E7000B084000F8F3FF1C08084036
:102CD000F0B590F818C0144E4FEA4C17BC592504B3
:102CE00018D4A30342F08053104D43F4004348BF6F
:102CF00044F0806443EA8143254043EA8C532B43EC
:102D0000BB51437EC28061F3010303F0F3036FF311
:102D100086134376007E0123054A83400020116814
:102D20000B431360F0BD00BF0009084000F833FCFE
:102D30001C0808404B790A79C97842EA0322437E8D
:102D400001F00301DB0601D5FFF7C2BFFFF78CBF1F
:102D5000427E017ED30602F003024FEA411148BFD2
:102D6000094BA2F1020258BF084B012A0B44196813
:102D700021F4001198BF41F080511960437E6FF338
:102D8000C30343760020704700090840000B084049
:102D9000F0B501F07F05EFF3118400238021EFF3FC
:102DA000108372B681F3118883F310888618F37C40
:102DB000C5B1062D21DC0121A9401940D1B1012561
:102DC000AC460CFA05F73942BE4610D023EA0E0392
:102DD000E4B2F37484F311881C236B4322B1603393
:102DE0001844F0BD1946E9E703F59273F8E7013599
:102DF000072DE6D1E4B284F311880020F1E710B585
:102E0000C0B1B9B1EFF3118200238024EFF3108336
:102E100072B684F3118883F310884B7E097EC3F366
:102E20000013184401238B40C17C0B43C374D3B2FD
:102E300083F3118810BDFFEC024B1868C0F30D201E
:102E4000704700BF08080840037C61F34103037426
:102E500000207047EFF3118000238022EFF31083EE
:102E600072B682F3118883F31088074A136839B168
:102E700023F002031360C3B283F31188002070476C
:102E800043F00203F6E700BF0408084008B540F02D
:102E90002000064B064A18601968890601D5013AD8
:102EA000FAD10320FDF73FFC002008BD10000840C8
:102EB000400D030008B51022064B1A60064A196837
:102EC000C90601D5013AFAD10320FDF72CFC0020F8
:102ED00008BD00BF10000840400D030038B503696D
:102EE00004460D4643B1437EDB0606D5007E8001D5
:102EF000FFF7CCFF23691BB938BDFFF7DBFFF9E70C
:102F000029462046FFF779FEF4E710B5EFF3118468
:102F100000238022EFF3108372B682F3118883F3CB
:102F200010886FF06D01E4B2FFF7D8FF84F31188C9
:102F3000002010BD084601F02BB910B5182001F093
:102F40002FF9044618B11822002101F04FFD204648
:102F500010BDFFEC70B5EFF3118500238022EFF375
:102F6000108372B682F3118883F31088037CDA062B
:102F70000ED50A4B1B68DB070AD5094E05203468BD
:102F800044F0010324F00104336001F0DDF8346003
:102F9000EDB285F31188002070BD00BF080808401D
:102FA00004080840054B064A1A6002F1604202F626
:102FB000E822136843F0044313607047100B084085
:102FC00018000860F0B5057E204F6D01EB5903F045
:102FD0000043002A33D0C688541E3444B4FBF6F4B0
:102FE000467E134306F0030643EAC443012E184EFF
:102FF00008BF43EA4473EB51457E047E05F00305A8
:103000006401012DA35907D1124D2D68ED0554BF60
:1030100043F0805343F0005323F08043033243F0E6
:1030200004439210A351037E00201B0303F180434D
:1030300003F50123824201EB800402DCF0BD012490
:10304000CEE7246801301C60F4E700BF1009084097
:103050000009084008080840F8B50D6907460C4605
:103060005DB90B7E2E495B015A5842F000625A50FE
:10307000637E65F382036376F8BDEB881BB94B7EF4
:1030800043F040034B762A89EB889A4202D3617E53
:10309000490638D59B1A627E002B6FF38612627642
:1030A0001ADDE6889E4217DC06D12B79DB0703D5B3
:1030B000D3B243F040036376217E1A4B4A01D258C3
:1030C000F31C92B2B2EBA30F08DA174A012310687F
:1030D0008B4003431360CFE71E46EDE72B89324652
:1030E000296820461944FFF76DFF637E43F004030F
:1030F0006376237E23B97B7C052262F307137B74FE
:103100002B891E442E812A89EB889A42B4D3617E92
:1031100011F04001B0D12046BDE8F840FFF76DBD89
:1031200000090840180908403408084030B5034633
:103130000A4C1A1A914200DC30BD22680433C2F3F3
:10314000072503F8042C03F8035CC2F30745C2F318
:10315000076203F8025C03F8012CEAE7001008405C
:10316000002882B006DD0023034904330A68984230
:103170000192FADC02B070470010084070B50546B5
:103180000C4622695AB9237E1A485B01195841F04E
:1031900000611950637E62F38203637670BDD1884B
:1031A00019B92046FFF729FDEBE7E388124E5A1EB6
:1031B0001144227E91FBF3F152014B43905943EAB3
:1031C000C1430C4900F0604003439351237E5B01EF
:1031D0005A5842F004425A50637E43F00403637627
:1031E000237E002BDAD16B7C062262F307136B740B
:1031F000D4E700BF000B0840100B08401A4B0246F2
:1032000070B5C0688B60EFF3118500238024EFF365
:10321000108372B684F3118883F31088537E13F001
:1032200008031DD114694B613CB9537E13F00406A9
:10323000C2E9041109D0204603E0506941611846F3
:103240005161EDB285F3118870BD13F01004114681
:1032500003D0FFF701FF3046F3E7FFF78FFFEAE700
:103260006FF00F00EDE700BF000089FF044B1A6804
:1032700042F400721A601A681207FCD5704700BF4A
:103280000408084038B5437E0446DD0639D5037E80
:1032900033495B015B58180431D5EFF311850023E6
:1032A0008022EFF3108372B682F3118883F31088C3
:1032B000227E5201535823F4004343F0904353506D
:1032C000237E284A5B01981801688907FCD5995824
:1032D00041F002019950207E8001FFF7D7FD22497D
:1032E000207E01220B68824023EA02030B606FF00C
:1032F0006D012046FFF7F2FDEDB285F31188002045
:1033000038BDEFF3118500238022EFF3108372B6EE
:1033100082F3118883F31088FFF7A8FF027E134918
:103320000A205201535823F4004343F09043535072
:10333000FDF7F9F9237E0E4A02215B010A489950F4
:10334000A2F54172136843F480631360227E036820
:1033500002F1100101228A4023EA02030360C6E75A
:1033600000090840080908401C080840000B0840F4
:10337000080B0840002210B5044611466030FFF7E4
:1033800021FE637C042262F307136374BDE81040DE
:10339000FFF708BE10B50446FFF768FF027E0A205B
:1033A0000A495201535843F0804343F400135350E9
:1033B000FDF7B9F9064A0020136843F480631360EF
:1033C000637E43F00803637610BD00BF000B084026
:1033D00004080840427E0346D20601D4FFF7DABF54
:1033E000027E06485201115841F40011115000208C
:1033F0005A7E42F008025A76704700BF0009084022
:1034000010B5EFF3118400238022EFF3108372B61E
:1034100082F3118883F3108829B1FFF799FCE4B295
:1034200084F3118810BDFFF7D5FFF8E710B50269E6
:10343000044622B9437E62F38203437610BD002125
:10344000FFF7DBFB637E6FF3820363765B07F5D4E4
:1034500021460248BDE81040FFF790BE840D0024CD
:10346000364A00202DE9F0471368354C23F001035C
:103470001360FFF70BFDE06818B103682146DB68B5
:103480009847DFF8C4A0FE23DFF8C88000270AF1C0
:10349000C409E37423751C26FF236FF06D0108F146
:1034A00020087E43013748F8203CA519C8F8E031D0
:1034B0000AEB0600FFF712FD95F879306FF06D0109
:1034C00009EB060003F0F3036FF3861385F87930F8
:1034D000FFF704FD95F83D31072F03F0F3036FF379
:1034E000861385F83D31D6D1164B4FF0FF320021BF
:1034F00015481A604FF001125A600B23134A1360EB
:1035000042F8043C52F8143C23F4FE6342F8143CA5
:103510004022637C6FF303036374237C6FF38203A5
:10352000237402232372FFF7D3FB402200210848B3
:10353000FFF79AFBBDE8F047FFF734BD04080840E9
:10354000840D002418080840E40D002414080840E5
:10355000A80E0024080908402DE9F843044600F5A8
:1035600092756FF0460104F160072846FFF7B6FC3C
:103570006FF046013846FFF7B1FC94F83D31032265
:10358000607D6FF3C30310F0600F84F83D3194F851
:1035900079306FF3C30384F87930237C6FF3000331
:1035A0002374637C62F30713637405D004F115017F
:1035B0002046FFF740FB71E0A27EE17D94F8188081
:1035C000637E94F81CE041EA082843EA0223E27E85
:1035D0000FFA88F81BB242EA0E2294F816E01FFA9E
:1035E00088FC9EB2BEF10C0F2AD80FF2080959F8D8
:1035F0002EF000BF29360008FF36000841360008CB
:103600005937000841360008FF37000855380008D0
:10361000553800085D38000881380008AD350008CD
:10362000AD3500089D360008217C11F0040F07D04D
:10363000022A05D110F0800F02D0BCF1000F04D097
:10364000237C43F00103237428E000F01F000128CD
:1036500050D044D30228F3D103F07F03062BEFD8D8
:10366000C3EBC30332064FEA83034CBF603303F559
:10367000927323445B7E13F008032ED163770222FA
:103680000023A37704F11D013846FFF79BFC637C00
:10369000042262F307136374FFF784FC237CDB07C7
:1036A00016D594F8783028468A495B015A5842F476
:1036B00000125A5094F8793043F0080384F87930B6
:1036C000FFF768FE237C43F001032374FFF76AFCD5
:1036D0000023A4F85E30BDE8F8830123CEE7002E76
:1036E000AED1C1F30013C1F34001A67741EA430113
:1036F0006177C7E784F81DC084F81EC0C2E7217C4B
:103700004F079DD5002A9BD100F01F00022817D13A
:10371000BCF1000F7FF44AAF03F07F03062B3FF6A6
:1037200045AFC3EBC303980033064CBF603000F5D0
:1037300092702044FFF70CFB2046FFF71BFEADE71D
:1037400000287FF433AFBCF1010F7FF42FAF0B469D
:1037500062F304132374EFE7217C4F077FF570AF0A
:10376000002A7FF46DAF00F01F00022813D1BCF1D6
:10377000000F40D103F07F03062B3CD8C3EBC303FB
:1037800032064FEA83004CBF603000F5927020444F
:10379000FFF720FED0E770BBBCF1010F03D141F071
:1037A00010012174C8E7BCF1020F24D116F0FF0FFD
:1037B00021D1360AA37C013E042E14D8DFE806F09E
:1037C000030B0D0F1100012262F30303A374237C8A
:1037D00043F02003BEE70222F6E70322F4E70422C7
:1037E000F2E70522F0E76FF30303A374237C43F0B1
:1037F00001032374EBE70B077FF522AFD6E6C7067C
:103800007FF41EAF002E7FF41BAF002A7FF418AFA9
:10381000BCF17F0F3FF614AF637C03F00F03022B64
:103820003FF40EAF2C4A136823F4FE6343EA0113FE
:103830001360637C227C31B1012161F30303637463
:1038400042F0040386E761F303036374134661F3F4
:1038500082037FE7C0067FF4F3AEA7E6237C590717
:103860007FF5EEAEC3067FF4EBAEBCF1000F7FF444
:10387000E7AE002E7FF4E4AE012A7FF4E1AE95E6D8
:10388000237C5F077FF5DCAEC1067FF4D9AE002E46
:103890007FF4D6AE002A7FF4D3AE04F115012046A2
:1038A000FFF7C9F900287FF4F9AE18F0FF0F637C29
:1038B000227C06D0022161F30303637442F0080303
:1038C000C1E6012161F303036374134666F3C30386
:1038D000B9E600BF00090840000808402DE9F04F94
:1038E00085B08D498D4B0C681B688D4A03EA040036
:1038F0001C4002EA00020A6000F0AB8026030ED5ED
:10390000884B894A1D68126815402D0C40F0AC8028
:103910001B68FF21854A1B0C002B40F09E8067032B
:103920000FD5804B804A1E6812681640B6B2002E32
:1039300040F00C811B68FF217D4A9BB2002B40F0B8
:10394000E580002C10DA7B4A01217B4D1368284664
:1039500023F001031360FDF767F9E86820B10368FD
:103960005B690BB12946984721050AD57249C86899
:1039700018B103681B6903B1984700216E48FDF731
:1039800053F9E2065FD56D4B1D6805F00F07062F52
:1039900059DC05F4F013B3F5002F00F08481B3F582
:1039A000402F00F08D81B3F5802F4CD1C5F30A155F
:1039B000002D48D0604B1C2606FB07369946D6F8EA
:1039C0003481B8F1000F40F0568196F83CB1BBF15C
:1039D000000F40F04C81D6F82C8198F8113003F09C
:1039E000F003102B40F04381402D2B4608F11D00C1
:1039F000A8BF40231FFA83FA00935146FFF796FBB6
:103A0000009BE81AFFF7ACFB96F83D3102226BF3FE
:103A1000820386F83D3198F81130A8F85EA062F371
:103A2000071388F8113003F0F003202B02D1404631
:103A3000FFF792FD1C2303FB079393F83D216FF3DF
:103A4000820283F83D213E4B1C4200F05181FFF77A
:103A500007FD002005B0BDE8F08FDD0701D5106837
:103A600011605B08203257E70026DFF8C080DFF8DE
:103A7000D8A0DFF8C4B0E80737D54FEA461959F89F
:103A80000870DAF800301F40F9071BD5012316F043
:103A9000FF0049F808309BF811302BD103F0F003F8
:103AA000602B0FD12748FFF7C1FC9BF83D3113F085
:103AB000040107D1FFF776FA9BF8113061F3071381
:103AC0008BF81130BA0702D5022349F808303B07BA
:103AD0000BD59BF8113003F0F003202B02D1584690
:103AE000FFF73AFD082349F808306D0806F1010692
:103AF000C1D114E703F00F03022BE3D11C2303FB16
:103B000000B000F59270FFF791FCDBE7DE0700D50F
:103B100011605B08203211E71400084018000840CB
:103B20000AFCB0F8180808401C080840080B0840B8
:103B30000809084004080840840D002420000840BB
:103B400000108000A80E0024140808400027F50784
:103B50007FD5754A4FEA471B744BDFF8E8A11B6815
:103B6000D2F800800122BA4012EA080F00925BF8F6
:103B70000A2018BF43F0800302EA030919F0010389
:103B800001933FD0009B5FFA87FC1C22684D28EA16
:103B90000308654B02FB0CF2C3F80080012302F11D
:103BA00060014BF80A302944687CBCF1000F56D103
:103BB00000F0F000502812D1284603920295FFF73A
:103BC0004BFADDE90232134493F8793013F0040123
:103BD00005D1FFF7E7F96B7C61F307136B742A7C5F
:103BE00090060FD553486FF34512AB7C016803F084
:103BF0000F0C6FF3030301F0700141EA0C11016037
:103C00002A74AB7419F0080F02D008234BF80A305D
:103C100019F0100F09D048481C2101FB070160383A
:103C2000FFF71AFA10234BF80A3019F0800F10D062
:103C3000019B5BB9009B1C213F4828EA03033A4AD9
:103C400001FB070160381360FFF706FA80234BF889
:103C50000A30760807F101077FF479AF71E600F0CA
:103C60000F000228CED12846FFF7F6F9CAE728460A
:103C7000FFF776FADEE6B8F80800B8F80660D8F87C
:103C80000030361A1844AE42A8BF2E46B7B23946A5
:103C9000FFF74CFAA81BFFF763FAB8F808301F4487
:103CA000A8F80870CFE6224B5B7C03F0F003102BE2
:103CB0007FF4C9AE214A136843F080631360C2E603
:103CC0001B4D082105F11500FFF730FA95F9153065
:103CD000002B0ADB2A7FEB7E53EA022305D06B7CA4
:103CE000012262F307136B74ADE66B7C0222F8E7E6
:103CF000A3047FF5F6AD124A1368A2F6F40223F48A
:103D0000FF6323F0070343F04003C2F8F438D2F80E
:103D1000F83743F48073C2F8F837136823F470530C
:103D200043F4C0531360DCE5340808401008084031
:103D3000840D002404080840E40D0024000B084012
:103D4000000908400809084038B50B4CE0602146DE
:103D500003681B689847054618B10023E3602846AE
:103D600038BD7520FCF7EAFD01212046FFF772F807
:103D700002232372F3E700BF840D0024F8B5074641
:103D8000EFF3118480260023EFF3108372B686F3DD
:103D9000118883F31088FFF763FBE4B284F3118882
:103DA0000E4D38463B6829465B689847EFF311840F
:103DB0000023EFF3108372B686F3118883F3108823
:103DC0007520E4B2FCF7A6FD00212846FFF742F873
:103DD0000020E86084F31188F8BD00BF840D002442
:103DE00070B5284DE86808B1FFF7C8FFEFF31186FA
:103DF00000238022EFF3108372B682F3118883F3DD
:103E00001088002400211F48F6B2FFF723F8752020
:103E10002C72FCF77FFD214622467520FCF7F6FF49
:103E2000FF23194A4FF4806013602032C2F8E0315A
:103E30001360C2F8003220321360C2F80032203220
:103E40001360C2F8003220321360C2F80032203210
:103E50001360C2F8003220321360C2F800324FF013
:103E6000FF320A4B1C605C605C62DC609A60FFF7AA
:103E70000DF8FFF71FF86B7C64F303036B7486F394
:103E8000118870BD840D00240809084010080840FE
:103E9000F8B5954B1A6822F0007242F080721A60F1
:103EA0001A685101FCD59148FEF74EF99048FEF78B
:103EB0004BF99048FEF748F98F4FFFF791FF8F4B72
:103EC0004FF4F472002118463E4600F08FFD8C49F5
:103ED000024603464FF01C0E4FF0400C42F8601BA8
:103EE0001C464260FE229866C27402750246C3F800
:103EF0002C0100200EFB00411C325764146591F820
:103F0000795045F0100581F87950C5B2013082F83A
:103F10005C5065F07F05072882F8485091F8795089
:103F20006FF3010581F87950A2F84AC0E2D100226E
:103F30001C274025D1B2C3F82461C3F830411C339B
:103F400083F8201183F80C1107FB0241013291F82C
:103F50003D01072A6FF3010081F83D01A3F80E51DE
:103F6000E8D1002267497520FCF750FF0028C0F215
:103F7000B7808022644D654B654F1A602A683E46C3
:103F8000644C42F040022A600320FCF7CCFB3B6803
:103F9000002B01DB013CF7D1012333605D4B32681C
:103FA000D20701D5013BFAD103200024FCF7BBFB6B
:103FB000594B4FF4803214201A6000F0C5F8574A6C
:103FC0003220136843F0C00313602B6823F00053C2
:103FD00043F080432B6000F0B7F8514B4FF4806002
:103FE0001C60A3F5C0631A68A3F2DC7322F4C0520C
:103FF000C3F8DC27D3F8DC2742F00302C3F8DC2740
:1040000040F201221A6002F592025A604932C3F866
:10401000E0204932C3F8E4204932C3F8E8204932AD
:10402000C3F8EC204932C3F8F0204932C3F8F42039
:10403000FEF72CFFFEF73EFF3A4B4FF0FF32FF2119
:104040001C60F03343F8EC4C43F8CC4C43F8E82CBC
:1040500043F8E44C344A186820330028B4BF4FF0CA
:104060000840002043F8200C43F8104C43F8181C7B
:104070009342F0D12D4B0022FF202D491C682033A4
:10408000002CB4BF4FF00844002443F8204C43F800
:10409000102C43F8180C8B42F0D1264926480A60B0
:1040A0004FF0FF32254B1A600268254B22F07F4209
:1040B00022F47C0222F47C4222F0FF02134381228C
:1040C0000360204B0D480B600021104B1A60FEF777
:1040D000C1FEFFF7C5F97520BDE8F840FCF72EBC1E
:1040E000BDE8F840FFF77CBE0C4802580BAC080056
:1040F0000CAC08000AAE0900BC9C0008840D00242A
:10410000A09C0008DD3800080C00084008000840AA
:1041100010000840400D030038000840000008402F
:10412000000E084010080840E0090840000B084055
:10413000E00B084018000840140008400400084044
:104140000AFCB0F810380C0082B0002345F261611F
:104150000093009A824201D302B070470193019A02
:104160008A4203D9009A01320092F2E7019A0132A1
:104170000192F4E708B50A460146034800F056F8F4
:10418000024B186008BD00BFD89C00086C0F0024CB
:10419000024B0146186800F0C0B800BF6C0F002445
:1041A000024B0146186800F016B900BF6C0F0024DE
:1041B000024B0A460146186800F06CB96C0F0024E7
:1041C000024B0146186800F0CFB900BF6C0F002405
:1041D000F8B50D461646044600F055F8AA1905F143
:1041E0000F036168082523F00F0322F00F024FF040
:1041F0000047D01A01441038C4E90113194641F8A8
:10420000085BA66877609860A2F108004D60E060E6
:10421000204642F8085C9B68E2683B43536000F02C
:1042200054F82046BDE8F84000F04DB801F10F0306
:1042300070B5A2F5A27423F00F034FF4A2720C44E0
:10424000184600211D46E41A03F5A27600F0CEFBC5
:10425000034600F1200200F5A0719A61A2F110005E
:1042600010321033D8618A42F7D1284600F007F89F
:10427000284622463146FFF7ABFF284670BD012293
:10428000002100F0C0BA10B50446FEF755F9C0B9D8
:1042900004F0C6F9002814DB04F04CF850B12046B5
:1042A00004F0E8F8C043C00F10BD00F09CF90368AB
:1042B000002B04DD204604F0A9F80028F5DB0120DE
:1042C000F2E70020F0E704F01BB938B505460868AE
:1042D0000C4600F015F8421C05EB021205EB001528
:1042E000AB6923B1196811B12068814205D394608C
:1042F000C4E9023203B1DC6038BD1A469B68F0E7BE
:10430000B0F5800F07D203090020012B00D87047B9
:1043100001305B08F9E71220704770B505460C467E
:10432000A9B1FFF7B0FF98B9EFF311830022802104
:10433000EFF3108272B681F3118882F31088D5F8FA
:104340004021DBB22260C5F8404183F3118870BD83
:1043500054F8043CA4F1080123F0004344F8043C61
:1043600054F8083CCA185068002814DBCB58D2E92E
:10437000026013448660906808B1D668C66012680F
:1043800054F8080C104444F8080C5A6802F0004233
:1043900002435A601A4654F8043CCB1A5868002865
:1043A00011DBD3E902018860996809B1D868C86057
:1043B000196854F8080C08441860516801F000416D
:1043C0000143516019462846FFF77FFF2846BDE8A4
:1043D0007040FFF778BF70B506460C46EFF31183C7
:1043E00000228021EFF3108272B681F3118882F3EC
:1043F00010880022D0F84011DBB2C0F8402183F3CE
:10440000118800293AD1002C36D004F1170525F087
:104410000F05AC423CD83046FFF735FFB5F5800FAD
:1044200032D22846FFF76CFF06EB0010846904B314
:104430002268A368AA4229D3E2689360A3680BB1FB
:10444000E268DA602368581B0F280CD923446119ED
:1044500060514D6025605A6802F0004202433046C8
:104460005A60FFF732FF6368083443F0004344F8B2
:10447000043C3046FFF727FF204670BD0D683046EC
:10448000FFF74BFF2946BCE71220CDE71C46CEE7DD
:104490000C46F1E7334B99422DE9F04707461646A3
:1044A00002D90020BDE8F0874D4205EA010A8A459D
:1044B000F7D1BAF1100F04D81146BDE8F047FFF765
:1044C0008ABF02F10F034FEA4A0123F00F03C91814
:1044D0002CBF012200229E428846E2D8002AE0D169
:1044E000FFF779FF81460028DBD00AF1FF34384618
:1044F000FFF7C9FEA9F108014C442C40A14523D087
:10450000A4F1080559F8083C6A1A0B440F2A9EBF0B
:104510005444A4F108056A1A581B286042F0004070
:10452000686049F8082C4A6822F000424A605A68DC
:10453000286802F00042024338465A602B68A3F113
:104540000808FFF7C2FE294606F1170222F00F0203
:10455000904502D9384600F013F83846FFF7B3FE0D
:1045600020469FE7FEFFFF7F38B50D46FFF733FF7C
:10457000044618B12A46002100F038FA204638BD1A
:10458000F0B40D680B4606464C19616800291ADB29
:104590005F59D4E9020127448860A16809B1E06845
:1045A000C860186899185C59801A204498504A606D
:1045B0001A6078689B5800F00040184378603046D5
:1045C000F0BCFFF782BE02F110018D4209D39918A9
:1045D000AD1A9D504A601A609B5843F000436360D7
:1045E000EEE7F0BC704708B500F08CFA143008BD57
:1045F00038B5012204460021283000F004F94FF0BC
:10460000FF35002304F12C002563C4F80431C4F8FD
:10461000083100F031F804F17400A56700F02CF8BF
:10462000C4F8C05004F1BC00BDE8384000F024B824
:1046300038B504462830FCF742FF0023C4F808319F
:10464000D4F804516DB904F13400FCF738FF04F1DB
:104650007C00FCF734FF04F1C400BDE83840FCF7EF
:104660002EBF284650F8083BC4F80431FCF727FF5A
:104670002846FFF78DFDE3E710B50122044600212F
:10468000083000F0C0F84FF6FF7363810023E36049
:1046900010BD70B5044603F0C3FF0546B4F90A30F7
:1046A000834209D004F10806304603F0AFFE00282B
:1046B000FADB6581012301E0E3680133E36070BD4B
:1046C000C368012B02DD013BC36070474FF6FF73E7
:1046D000083043800023436003F012BF00230360CF
:1046E0000B6813B90860486070474B681860FAE7B8
:1046F0000B6893B188B1834209D11A680A604A688D
:104700009A420AD100234B60704713462AB11A68B7
:104710008242FAD1184600F00BB8704703682BB1FB
:104720001A68026002B9426000221A601846704797
:104730000A68036852B14BB14A689A424FF00002CE
:1047400015BF19684860016002601A60184670471A
:10475000002303604B6843600B6813B9086048602E
:1047600070474B681860FAE7002343600B680360EA
:104770000B6813B9C1E900007047586008607047C2
:10478000D0E9003232B90B6033B94A600023C0E986
:10479000003370471360F7E75A60F7E70F4C904615
:1047A000064622682DE988480F4652B90C4DDFF8BD
:1047B0003490DFF834A0DFF834B04D4506D1012342
:1047C000236041463846B047FCF7B6FD55F8043B38
:1047D0005345F2D35B45F0D29847EEE7700F0024C3
:1047E00038A0000838A000080000000838A0000821
:1047F00030B1B2F5004F03D212B2028000207047F0
:104800006FF01500704708B530B1B2F5004F03D214
:1048100012B20280002008BDFFF7E5FE16230360F8
:104820004FF0FF30F7E71F299FBF012303FA01F183
:1048300003680B439ABF036000206FF015007047B8
:104840001F299FBF012303FA01F103688B439ABF1D
:10485000036000206FF015007047002303601846C6
:1048600070471F299DBF0068C84000F001006FF02D
:10487000150070470FB413B504AB53F8044B019304
:1048800003F050FD019A21464C3000F06BF802B065
:10489000BDE8104004B0704770B50646C0B100F0E6
:1048A0003DF90025D6F8DC4024B9304600F03EF949
:1048B000284670BDB4F840309B0707D5012120463B
:1048C00000F008F835EA200528BF05462468EBE724
:1048D0000546EDE7F8B5436805460F46002B3EDB7D
:1048E000B0F840309B073AD5FFF7D3FE2C69FCB1F6
:1048F000AE69B44207D12846FFF7E2FEAC692B69E6
:10490000E41A2046F8BDEB699C4226D1361B32469C
:104910002146686803F06CFB00280DDA95F84230F8
:1049200043F0020385F84230FFF75DFE04686442FD
:104930002846FFF7C5FEE4E70444361A0FB1002EFF
:10494000E5DC2B692644AB61B442D4D0AB695A1C78
:10495000AA6114F8012B1A70F6E70024E8E76FF05B
:104960000804CEE77FB5044616460D460146684664
:1049700000F026F82046FFF78CFE294632466846AE
:1049800000F0D8F805462046FFF79AFE284604B006
:1049900070BD0121C068FFF79DBF38B504460D46C4
:1049A000E168284600F0B2FD013003D0A36801336E
:1049B000A36038BDFFF717FE0368042BF0D0F8E7BB
:1049C000074B03600B694BB1B1F84030DB0505D4F0
:1049D000044B43600023C0E902317047024BF8E703
:1049E0009B49000893490008314B00082DE9F0432A
:1049F000B2B3C70703463ED5013A03F8011B012AAB
:104A00002CD941EA01259E07ADB231D0023A23F8F4
:104A1000025B032A1DD95C0745EA054C4FF00008EC
:104A200016BF141F144643F804CB48EA0C06674629
:104A3000224603EB040E072A14D8E2086FF007069B
:104A400006FB02423440032A234484BF043A43F85D
:104A500004CB012A02D9023A23F8025B02B1197091
:104A6000BDE8F083AEEB0208083AC8E90067E2E768
:104A7000032AD0D8EFE7012AC3D8F0E7421E11F885
:104A8000013B02F8013F002BF9D1704703461A7829
:104A9000591C0AB9181A70470B46F8E70244013945
:104AA000034610B5934207D011F8014F03F8014BAC
:104AB000002CF7D1934200D110BD03F8014BF9E768
:104AC00000220E4B30B59C18D55864688C4209D131
:104AD000C561836823F4805323F00F03234383606D
:104AE000002030BDA94201D1C161F2E70832F82AA5
:104AF000E9D1C1614FF48054EBE700BFE09C0008AE
:104B0000C06970471FB5002001A903F025FC0028EB
:104B1000ACBF0298002005B05DF804FB10B5044658
:104B2000204603F073FC0028FADB10BD03F0E8BC5C
:104B3000002070472DE9F04F05468DB092460024C5
:104B40004B1C91F800800293B8F1000F00F0EF8346
:104B5000B8F1250F06D191F801808B1CB8F1250F13
:104B6000029307D12B684146284601349847CDF877
:104B700004A0D9E300270A223E46B946B9F13F0F07
:104B80004FD8B8F12B0F41D014D8B8F1200F3FD037
:104B9000B8F1230F42D0A8F13003DBB2092B53D870
:104BA00019F4807F12BF02FB073749F0800902FB2E
:104BB000063607E0B8F12D0F2DD0B8F1300FEAD14D
:104BC00049F00109029B13F8018B0293B8F1000F21
:104BD000D4D1A8F14503022B7CD808F1200849F470
:104BE00000595FFA88F819F4807F08BF0627B8F1EA
:104BF000650FFAB240F09280013249F48049D2B296
:104C00000F2A28BF0F22114600228EE049F0020928
:104C100049F00409D6E749F00809D3E749F010093B
:104C2000D0E7B9F5007FB6D3B8F17A0F2DD0B8F13F
:104C3000740F2AD0B8F16A0F24D129F480691FFAC1
:104C400089F949F42069BDE7B8F12A0F10D119F4A8
:104C5000807F5AF8043B02D023EAE377B2E7002BC7
:104C6000A7BF49F080091E465E4249F08809A9E7BE
:104C7000B8F12E0FD8D119F4807F40F0588349F451
:104C800080799FE7B8F16C0F0BD119F4007F18BF42
:104C900049F4006929F480691FFA89F949F4007917
:104CA00090E7B8F1680F0BD119F4806F18BF49F481
:104CB000006929F400791FFA89F949F4806981E7CC
:104CC000B8F1700F02BF29F420691FFA89F949F47D
:104CD00000797EE7A8F16503022B84D9B8F1630F50
:104CE00000F0A481B8F1730F03D0B8F1530F40F076
:104CF000C5810AF10403DAF800A00193B64BBAF1BA
:104D0000000F08BF9A4619F4807F504614BF3946F9
:104D10004FF0FF3100F018FC074691E1B8F1660F43
:104D20007FF46EAF49F400490F210AF1070A06A883
:104D30002AF0070A0AF108039AED000B019300F02C
:104D40001FFB9DF81C3003F00902012A3CD019F02A
:104D5000020F3CD119F0040F14BF4FF020084FF0A0
:104D6000000813F00C0F3ED0B8F1000F0CBF032366
:104D70000423B3420CDA19F0080FA6EB030608D19E
:104D800037462B68202128469847013FF9D1344403
:104D90000026B8F1000F04D02B68414628460134A4
:104DA00098479DF81C3009F400598C4F13F0080FF8
:104DB0008B4B08BF1F46A4EB070808EB070417F846
:104DC000011B39B93746ACE24FF02D08C9E74FF067
:104DD0002B08C6E7B9F1000F01D02039C9B22B6802
:104DE00028469847E9E77F4B5FFA80FBDDF818A07B
:104DF00019EA030F5A461AD10BF1050306A90B4411
:104E0000BBF1000F03D013F8011D302928D01AF18F
:104E1000040F2ADB924528DABAF1000F49F4004961
:104E200001DBDA4524DA0AF10107ABEB07070FFAD9
:104E300089F3002B0393B6BF2AEAEA7305230133F3
:104E4000B8F1000F00D00133A7B17A1C1344B3426C
:104E5000B4BFF61A002619F0090F1BD1334614E02F
:104E60000BF1FF3B5FFA8BFBCAE70BF1FF37DEE785
:104E70000027DCE719F0100F18BF0133E7E7202106
:104E8000284604939047049B013B2A68002BF6D1E7
:104E900034441E46631C2A680493B8F1000F04D002
:104EA000414628469047049B1C4619F0080F0CD138
:104EB000B04604E008F1FF383021284698472B68B7
:104EC000B8F1000FF6D134444646039B002B48DA74
:104ED0002AEAEA787B42AAEB08020493B8F1FF3F82
:104EE00004F1010706D12B682E21284603923C4687
:104EF0009847039A5A4508F1FF38049936BF06AB24
:104F000030279B1802F1010238BF5F79631C884586
:104F100003932B681CDA19F0100F06D0B8F1FF3F8D
:104F200003D12E2128469847039CC2450AD19DF8FB
:104F30001D30352B13D805D19DF81C3013F0100F00
:104F400008BF312701342B6839462846984739E78E
:104F50003946284605929847039C059ABEE73127B3
:104F6000F0E79DF81D10284631291EBF9DF81C3022
:104F700023F010038DF81C302B689847002F2B6806
:104F800043DD02344FF001082E212846984747455B
:104F90002B6829DA19F4005F2B6828460CBF6521BD
:104FA00045219847BAF1000F04DB38D19DF81C3039
:104FB000DB0634D5CAF1000A2D212B682846984714
:104FC0003021BAF1090F2CDC2B68284698470434AD
:104FD0002B680AF13001B8E7D89D0008E39D00086E
:104FE000DF9D000800C0FFFFC345284604F101040F
:104FF0008ABF0CAA3021424408F1010888BF12F888
:10500000131C5FFA88F89847C1E719F0100F01D117
:105010000134BFE72E21284602349847BAE72B21F6
:10502000CBE70131AAF10A0AC9B2CAE70AF10403BF
:1050300001270193DAF800300DF1300A0AF8183D23
:1050400019F0080F0CD00AEB070813E0013E2B689B
:10505000202128469847BE42A8EB0604F6D8F2E77E
:1050600004EB0608F7E72B6828461AF8011B984757
:1050700006B1013ED045F6D13C44A3E6B8F1640F39
:1050800009F4206302D0B8F1690F78D1B3F5206F2D
:1050900061D10AF1070A2AF0070A0AF10803DAE9DE
:1050A00000010193002829F4805B71F100032BF0CB
:1050B000100B06DA40424BF4805B61EB41011FFAB2
:1050C0008BFB1BF4807F04D01FB950EA010300F072
:1050D000B6800DF118090A234A4600F02DF9A0EB1D
:1050E00009095FFA89F91BF4807FC84600F0A9809E
:1050F0002BF0010AB9451FFA8AFA80F2A58044F222
:105100001002FBB20BEA0202102A03D12BF0110AA3
:105110001FFA8AFA1AF0100F00F0A3800CAA4A4472
:1051200012F8192C302A40F091802AF4C04A2AF053
:10513000100A1FFA8AFA1AF0080F40F0A3801AF03A
:10514000010F05D0B34280F2B780F71AF3B24F4493
:10515000A3EB040B91E0524619F4007F52F8043B94
:10516000019218464FEAE3719CD119F4806F99D0EF
:1051700019F4006F0CBF18B258B2C11792E7B3F51B
:10518000206F20D10AF1070A2AF0070A0AF1080362
:10519000DAE90001019329F0060BB8F1700F1FFA4C
:1051A0008BFB3FD022D8B8F1580F3ED0B8F16F0F2B
:1051B00043D02B6828462521023498472B68414666
:1051C00028469847B0E00AF1040319F4007F0193E0
:1051D000DAF8000001D00021DDE719F4806FFAD081
:1051E00019F4006F0CBF80B2C0B2F4E7B8F1750FCC
:1051F00009D0B8F1780FDCD11BF0100F01D04BF4BF
:10520000804B102304E029F0160B0A231FFA8BFBB6
:105210001BF4807F03D017B950EA01020FD00DF1C3
:10522000180959E74BF0100BE6E719F0100F01D001
:105230004BF4C04B4FF40473EAE70823E8E7B946A0
:1052400051E74B46DA4665E74B4663E71AF4804F71
:1052500002D103F1010B01E003F1020B5FFA8BF3C2
:1052600069E741F206021AEA020F3FF464AFF0E781
:105270002B6820212846013498470BEB0403DBB24E
:10528000B342F5DBB342B4BFF61A00261AF0100F92
:1052900014D02B683021284698471AF4804F2CD020
:1052A0001AF4005F04F102042B680CBF7821582126
:1052B00028469847274418E04F4649E741F206033D
:1052C0001AEA030FF6D01AF0020F04F101042B685A
:1052D00014BF2B2120211AF4805F18BF2D21E7E78E
:1052E0002B6830212846013498473B1B4B45F7DC9F
:1052F000B9F1000F03D1444464E50134DAE709F160
:10530000FF390CAB28465FFA89F903EB09022B68D9
:1053100012F8181C9847EBE7013F2B68202128461C
:105320009847002FF8D13444DDE901A108E4204674
:105330000DB0BDE8F08F00BF2DE9F84313F40077FE
:1053400016461CBF23F4007301271C46DD172246B6
:105350002B4603F077FD092A8046894608DC303267
:1053600058EA090306F8012BF1D13046BDE8F8836D
:105370000FB13732F4E75732F2E7FFECC2925D7DAE
:105380002DE9F74F10EE904A07460E4614F0004400
:105390001CBFB1EE400B0124B5EE400BF1EE10FA4C
:1053A00014D144F00204421D00233021B34209DB32
:1053B0000025BB19002230465A713C713D6003B094
:1053C000BDE8F08F02F8011B0133EFE7B4EE400BAC
:1053D000F1EE10FA02D744F00804E9E7B0EEC07B22
:1053E0009FED3F6BB4EE467BF1EE10FA02DD44F028
:1053F0000404DDE79FED3C7BB4EEC70BF1EE10FA41
:1054000058D53F4908230F2501209FED396B31ED19
:10541000027B20EE077BB4EEC67BF1EE10FA05D5D9
:1054200000FA03FCB0EE470BA5EB0C0513F1FF33BC
:10543000EDD232B125EAE57301331A449642A8BF92
:105440001646304B03EBC60393ED007B30EE070BA3
:105450009FED277BB4EEC70BF1EE10FA04DBB2EE42
:10546000047B013580EE070B07F1050B4FF0000AB6
:105470000FF28409D9E9008951EC100B03F0FCFC10
:10548000CDE90001564594DD42464B460AF1010A3A
:10549000DDE9000103F0D6FC303049460BF8010B82
:1054A0004046CDE900230A22002303F0CBFC8046CE
:1054B0008946E7E7144908230F25012031ED026BE7
:1054C00020EE066BB4EEC76BF1EE10FA04DB00FAC7
:1054D00003FCB0EE460B654413F1FF33EED2A8E7B0
:1054E000FFFFFFFFFFFFEF7F00003426F56B0C434B
:1054F0000080E03779C341430080C6A47E8D03005D
:10550000F89E0008E89D0008B09E000837B50446E4
:1055100002A80A460D4600F8014D012100F020F8CE
:10552000002804DC4FF0FF34204603B030BD0A2CC5
:10553000FAD195F842305B07F6D501212846FFF7EE
:10554000C9F90028F0DAEDE70346014410B58B42B3
:1055500002D01A785C1C0AB9181A10BD2346F6E767
:105560002DE9F04107460E46154642B9FFF73BF8D4
:105570004FF0FF34092303602046BDE8F081B2F804
:1055800040309B0706D4FFF72EF8092303604FF045
:10559000FF3418E013693BB90A460146686802F017
:1055A00027FD041EE8DAF2E71046FFF772F82846F6
:1055B00000F034F800282FDA4FF0FF342846FFF7C8
:1055C0007FF8002CD8DA95F8423043F0020385F8D2
:1055D0004230D1E7D5E905329B1A511EB34228BFAC
:1055E0003346F61A04EB0308444509D113446A69AB
:1055F0009A42AB6109D94446002EEBD1E41BDDE7AA
:1056000014F8010B01F8010FEEE700212846FFF71F
:1056100061F90028EFDACFE73C46EDE710B5044624
:1056200030B9FEF7E0FF092303604FF0FF3010BDF3
:105630000369F3B1FFF72DF8E0692269904213D0B6
:10564000A36994F843101B1A2046C4E906220022DD
:10565000591A84F84320012200F00DF8002803DADB
:105660002046FFF72DF8E0E72046FFF729F8002055
:10567000DDE71846DBE770B504460D461646FFF732
:10568000CDFF002802DA4FF0FF3070BD204600F059
:1056900010F80028F7DB002332462946606884F8BA
:1056A000433002F094FB01304FF0FF3018BF002070
:1056B000EBE7026932B1B0F840309B0702D5012117
:1056C000FFF708B900207047022901D100F018BB8C
:1056D0007047FFEC08B5094B1B7813F0FD0F02D0A3
:1056E0004FF0FF3008BDC307FAD500F03FFB00289C
:1056F000F6DB034B02221A70F4E700BF750F00249B
:105700007C14002410B5084C606003F045FDFFF7E1
:10571000E1FF002804DB054A13680133136010BD64
:105720006368002BF1D1FAE780140024780F00247D
:1057300008B5FFF7E7FFA0F120035842584108BD24
:10574000034B1B78022B01D100F036BB704700BF22
:10575000750F002410B5124C236801331ED0114B75
:105760001A68053B9A4219D90F4B9B6803F10063F5
:1057700003F500339A4211D203F068FD03F036FDC1
:1057800000F0E8FA03F040FD03F008FD204603F0C6
:1057900077FD2046BDE8104003F01ABE10BD00BFE3
:1057A0000000020804000208860000240C4A0023BE
:1057B00010B5144652F8231021B152F823100139C4
:1057C00042F823100133042BF4D1064B1B7833B974
:1057D000A36823B9022003F0E9FD3223A36010BDC2
:1057E00080140024740F0024024BD860DA68002A69
:1057F000FCD17047801400242DE9F04FBF4F8FB0CB
:1058000000258146BE4EB8463D700295B46803F04F
:10581000D9FCDFF80CA3B9F1000F01D0CAF8009051
:10582000B84FCAF808503D704FF0FF35012003F023
:10583000B3FDB9F1000F04D0DAF80030002B00F00E
:105840003C820020FFF75EFF0390039B002BF0DB00
:10585000012003F097FD039B213B102BE6D801A20A
:1058600052F823F0A9580008BF5800083159000821
:105870002D5800082D5800082D580008C35900085D
:105880002D580008615A0008255B0008715B00086C
:10589000CF5B0008255C0008F55B00082D58000868
:1058A000975C0008835900080220FFF741FF002899
:1058B00000F01582029B43F00103029361E04FF474
:1058C0007A70FFF71FFFB0F1000BC0F208820220D0
:1058D000FFF72EFF002800F002820BF1FF300428B2
:1058E00000F2FD81DFE800F0030B0E11140004212B
:1058F0008548FFF725FF029B43F00203DDE7042103
:105900007F48F6E704218148F3E704218048F0E767
:105910004FF01C09484609F1040903F0D1FC0421A9
:10592000099009A8FFF70CFFB9F12C0FF2D1E2E7BB
:105930000220FFF7FDFE002800F0D181029B03F05A
:105940000303032B40F0CB8101234FF0000B022017
:105950003B7003F017FD03F084FC584603F096FCFF
:10596000044600BB0220387003F016FDB368A34262
:105970001FD8029B002443F004033C700293CAF832
:10598000084098F800301BB9624B1B7888F800304B
:105990000EA841F2120302214FF0000920F8143D35
:1059A000FFF7CEFE42E758460BF1010B03F074FC03
:1059B000D3E7204603F084FC013040F063810434D7
:1059C000D4E73220FFF79EFE031EC0F2888113F059
:1059D000030B40F084811A19B1688A4200F27F817A
:1059E000B3F5807F00F27B814B4A9B4516D1C820DE
:1059F000FFF79EFE002800F0728124B9464B4FF05D
:105A0000FF321D681A602BF0030B434BA3441B1B92
:105A10005C4516D1029B43F008034EE74FF47A70C1
:105A2000CDE90032FFF76EFE039003990029C0F222
:105A300056810399019A009B0BF802100BF1010BA0
:105A4000D3E719592046009303F034FC204603F0B5
:105A500037FC009B1A59904240F014810434D7E778
:105A60000220FFF765FE002800F039814FF00009A1
:105A7000CB4617E0B9F1000F21D1691C1FD0099561
:105A800026494B68B3B3002209A8135C013283EAAC
:105A90000B03042ADBB251F8233083EA1B2BF4D129
:105AA00009F10409B3684B45E4D80EA8042140F875
:105AB00028BDFFF745FE029B43F01003FDE6484674
:105AC00003F0FEFB0990DBE702F0010C5208BCF189
:105AD000000F07D082F06D4282F4380282F4034254
:105AE00082F020020138EFD141F823200133B3F5D1
:105AF000807FC8D01A460820E6E700BF750F002453
:105B000086000024740F0024F89E00088A000024F8
:105B10008E0000247C1400247C1300247C0F0024BD
:105B2000801400244FF0000B09AB64200093FFF7B2
:105B3000E9FD0028C0F2D380009B0BF803000BF1B5
:105B4000010BBBF1040FF0D1099B02200093FFF77A
:105B5000EFFD009B002800F0C280184603F0BAFB5E
:105B60000EAB594643F8240D1846FFF7E9FD08E748
:105B70004FF0000B09AB64200093FFF7C3FD002832
:105B8000C0F2AD80009B0BF803000BF1010BBBF1E1
:105B9000040FF0D1099B02200093FFF7C9FD0028F4
:105BA00000F09D80009B9A0740F09980082B00F23E
:105BB0009680184603F0E0FB0EAB594643F8200DE3
:105BC0001846FFF7BDFD029B43F0400375E6022037
:105BD000FFF7AEFD002800F0828003F07DFB0EABE6
:105BE000042143F81C0D1846FFF7AAFD029B43F061
:105BF000800362E60220FFF79BFD00286FD009A911
:105C0000142003F06FFB81460EA8042140F8189D74
:105C1000FFF796FD494609A8FFF792FD029B43F462
:105C200080734AE66420FFF76DFD002857DB5FFABA
:105C300080FBBBF11E0F52D80220FFF779FD002830
:105C40004DD04FF4D07003F03BFB00904FF4D27076
:105C500003F036FB274B009A9A4240D1264B9842DC
:105C60003DD1264B4FF4D0704BEA03031946009305
:105C700003F020FB4FF4D07003F022FB009B98420E
:105C80003FF47FAE0EA841F21213022120F8143D1A
:105C9000FFF756FDCAE54FF47A70FFF749FDF0B102
:105CA0006B1C0DD10EA841F21203022120F8143D05
:105CB000FFF746FD6420FFF797FD0FB0BDE8F08FBA
:105CC000029B03F01B031B2B09D12946002003F084
:105CD000F1FA002003F0F4FA8542D3D1E2E741F271
:105CE00012330EA8022120F8143DFFF729FD0023EE
:105CF00002939BE5FFECC2925D7D05C500ECC2926C
:105D000038B50F4B0F4C002808BF184602F0F0FFC3
:105D10000D49206002F0FAFF0C4B00B118604FF003
:105D2000FF320B4D432118682A6002F0F2F8002878
:105D300005DB28602068BDE83840FEF729BA38BD89
:105D4000E49B000894140024FC9E00089014002496
:105D50007800002410B5044C206801F0C0FE4FF01C
:105D6000FF33236010BD00BF7800002413B50F4C33
:105D70002368002B0FDA0E4B4321186802F0C9F894
:105D8000002803DA4FF0FF3002B010BD094B20604D
:105D90001868FEF7FDF901220DF10701206802F0F5
:105DA000F2F80128EED19DF80700EDE77800002415
:105DB0009014002494140024024B0A4601461868EB
:105DC00002F016B97800002403464FF60472084624
:105DD000934210B513D04FF60C72934212D04FF687
:105DE0000172934225D1FAF710FF002804461EDA0B
:105DF0006442FEF7F8FB04604FF0FF3010BD03F083
:105E0000C3FBF2E70B78012B05D14B78012B05D0B2
:105E10000DD3022B07D06FF01504E9E749688078AD
:105E200001F04AFBE1E74B68186801F0CDFB002068
:105E3000E4E76FF01804DBE770B504460D46A36B8A
:105E40002046DB6A98470028F9D0A36B29462046F4
:105E50005B6ABDE8704018472DE9F74F458C044652
:105E6000B0F9263089462DB24FF0800B01920135F2
:105E7000AB42D8BF0025A38C1BB2AB420AD0638CC7
:105E80002DB2A26A00201BB202F80390658403B011
:105E9000BDE8F08F019B002B30D0EFF31188EFF3BA
:105EA000108672B68BF3118886F31088A38C1BB210
:105EB000AB421ED1E27802F0FF0AE2B90121A26BE7
:105EC00020466170926A904704F1180002F066FA69
:105ED000A26B07465146926A204690475FFA88F8BF
:105EE00088F31188E37863B9002FC4DA6FF00300F8
:105EF000CDE70027F2E76FF07F07EFE76FF00A00CA
:105F0000C5E76FF07F00C2E72DE9F74F83680746CA
:105F1000884601925C6904F12C09484602F03EFA79
:105F2000051E1FDB00254FF0010B019B9D4204D293
:105F3000E378DBB10DB96FF07F05A36B012120463B
:105F40009B699847E28D238E12B21BB29A4206D10A
:105F5000A36B1B6A1BB10022204611469847484696
:105F600002F096FA284603B0BDE8F08F238EE28D4A
:105F700019B212B28A4220D0626B0133525C1BB25A
:105F8000B4F932109942D8BF00232386A36813F4D2
:105F9000E07F05D00A2A09D113F0400F18BF0D2267
:105FA00088F80020013508F10108BEE70D2AF7D175
:105FB00013F4807F18BF0A22F2E7002DBDD1BB6821
:105FC000002B4AD03D6815F0400549D1EFF3118A06
:105FD0008023EFF3108672B683F3118886F310885E
:105FE000A26B294620465FFA8AFA92699047E18DB2
:105FF000228E09B212B2914227D1A26B0121204612
:1060000092699047E18D228E09B212B2914202D07C
:106010008AF3118889E7E278A2B984F802B004F122
:106020001A0002F0BBF98AF31188002803DBE37839
:10603000002B3FF47AAFE378002B7FF47CAF6FF056
:1060400003057AE76FF07F00EDE78AF31188A36B11
:10605000012120469B69984767E76FF050056CE780
:106060006FF00A0569E72DE9F04183685C6904F186
:106070001608404602F092F9061E21DBE378002B59
:1060800034D12578013515F0FF0532D0012D2BD103
:10609000EFF311878022EFF3108372B682F3118839
:1060A00083F310882379FFB26BB9A36B20461B687A
:1060B0009847061E07DA87F31188404602F0E8F990
:1060C0003046BDE8F081A36B20469B689847061ECA
:1060D000A36B03DA5B6820469847ECE79B690121D4
:1060E0002046984787F311882570E6E76FF07F0612
:1060F000E3E76FF01706E0E7F7B50E4600F140055D
:1061000000F1500755F8044B8CB12379627943F0C4
:1061100018033340134363714BB101A9E06802F0E7
:106120005BFD019B002B02DCE06802F0B1F9BD428F
:10613000E8D103B0F0BD2DE9F843836888461546E1
:106140005C6904F11C07384602F028F9061E52DB90
:10615000002D53D004F14002002352F8045B002DBF
:1061600036D1103304F1200944F8238004EB830373
:106170004846C8F8103002F041F9638CB4F9262083
:106180001BB201339A42D8BF0023A28C12B29A42AA
:1061900027D1484604F12C0902F07AF9484602F06A
:1061A0002DF9E28D238E484612B21BB29A421EBFD1
:1061B00098F8043003F001031D4302F069F9E37815
:1061C000A3B145F0180529462046FFF795FF0FE0DB
:1061D0000133042BC1D100236FF00F06C8F8103033
:1061E00006E098F8045005F00405D2E7002DEAD146
:1061F000384602F04DF93046BDE8F883D8F8103043
:10620000002BF5D01D60C8F81050F1E72DE9F047DC
:1062100000F1200704468846384602F0BFF8051E04
:106220001DDBEFF3118600238022EFF3108372B69B
:1062300082F3118883F31088E37803F0FF0553B3EA
:10624000638C6FF07F05A384F6B286F311881E4B32
:10625000002D1E6899462CDA384602F019F92846B6
:10626000BDE8F087A36B012184F801A020469B6A5A
:106270009847484602F092F8A36B054600219B6AB6
:1062800020469847002DDFDB628CA38C12B21BB234
:106290009A42E7D1D8E74FF0010A04F11809F3E771
:1062A0004FF47A7002F082F9D9F800309B1B434515
:1062B00006D2A36B20461B6B98470028F0D0CBE793
:1062C0006FF07305CBE700BFA41400242DE9F0475D
:1062D00083680746884616465C69FCF72DF920B1AD
:1062E000E378ABB16FF07F0525E002F023F80028DA
:1062F000F6D104F1200A504602F050F8051E1ADBD0
:10630000E37803F0FF018BB3504602F0C1F8E9E7F0
:10631000EFF3118500238022EFF3108372B682F32E
:10632000118883F3108808EB0607474506D1EDB2C4
:1063300085F3118835462846BDE8F087E36818F8EC
:10634000011BD80703D50D2905D11A0705D420460E
:10635000FFF772FDE9E70A29F9D113F0240F03D002
:106360000D212046FFF768FD0A21F0E73F68B1469E
:10637000A36B204687F040079B6AC7F380179847B6
:10638000B9F1000F01D1354623E0E36818F8011B8D
:10639000D80703D50D290AD11A070AD43A46204650
:1063A000FFF75AFD051E10DB09F1FF39E8E70A295E
:1063B000F4D113F0240F01D10A21EFE73A460D2161
:1063C0002046FFF749FD051EF6DAB14501D2A6EBDE
:1063D0000905628CA38C12B21BB29A4204D0A36B43
:1063E000012120469B6A9847504602F051F8A2E7E7
:1063F0004FF6FF732DE9F0418B8207460B790C466F
:106400002BB10B6943F001030B610523CB60012223
:10641000002104F1200004F11806FEF7E9F9012239
:10642000002104F12C00FEF7E3F90122002104F120
:106430001600FEF7DDF90022304604F11A05114678
:10644000FEF7D6F9002228461146FEF7D1F90122BF
:10645000002104F11C00FEF7CBF90021304602F0C8
:10646000C5FB0021284602F0C1FB234638464FF405
:10647000DB720249BDE8F04101F033BE009F000825
:1064800010B504460121FFF737FEA3783BB1002386
:1064900004F11A00A370BDE8104001F0F9BF10BD6F
:1064A00010B504460421FFF727FE63783BB10023B3
:1064B00004F118006370BDE8104001F0E9BF10BDA1
:1064C00070B583680E4615465C69A36B1B699847D7
:1064D00010F1190F40F0B48040F219139E4200F001
:1064E000AB80B6F58D7F2DDA40F215139E4200F099
:1064F0009480B6F58C7F00F09780B6F58A7F47D1FF
:10650000EFF3118600238022EFF3108372B682F33B
:10651000118883F3108835F0020207D1E38D2386BA
:10652000A36B1B6A13B1114620469847013D012D0C
:1065300004D8638C2046A384FFF7B2FFF6B286F33B
:10654000118824E0B6F5427F2BD040F209339E42F9
:1065500043D040F207339E421AD1EFF3118100235A
:106560008022EFF3108372B682F3118883F31088D0
:10657000228EE38D12B21BB29A420ADCE38D228E88
:106580001BB212B29B1ACAB282F311882B60002090
:1065900070BD228EE08D12B2B4F9323000B2121A00
:1065A000F0E7EFF3118100238022EFF3108372B63E
:1065B00082F3118883F31088A28C638C12B21BB211
:1065C0009A4203DC638CA28C1BB2DAE7A28C608C4B
:1065D00012B2B4F9263000B2E1E7EFF311810023E3
:1065E0008022EFF3108372B682F3118883F3108850
:1065F000628CA38C12B21BB29A4206DAA38C628C14
:106600001BB212B29B1A013BBDE7628CA08C12B286
:10661000B4F9263000B2121AF4E7204642F21071A3
:10662000BDE87040FFF7F2BD002D22DBB4F9143055
:10663000002B1EDAA582AAE74FF6FF73A382A6E716
:106640000028A5D140F201139E420AD0B6F5817F01
:106650009ED175B12B68A3606B68E360EB68236122
:1066600096E735B1A3682B60E3686B602369EB6044
:106670008EE76FF015008BE770B504460E46EFF31A
:10668000118500238022EFF3108372B682F3118804
:1066900083F3108881F00103C37089B91821FFF7D3
:1066A0002BFD637823B1667004F1180001F0F0FE51
:1066B000A3782BB1002304F11A00A37001F0E8FEC7
:1066C000EDB285F3118870BD10B504460021183075
:1066D00001F023FF002104F11A0001F01EFF012147
:1066E00004F1200001F019FF012104F12C0001F058
:1066F00014FF04F11C000121BDE8104001F00DBFA2
:1067000070B5836806465C6904F11605284601F0F9
:1067100075FE2378012B06D9013B2370284601F032
:10672000B7FE002070BD0021A36B204621709B693D
:10673000984733685B0604D44FF47A612046FFF72C
:1067400065FDEFF3118600238022EFF3108372B60C
:1067500082F3118883F31088A36B2046DB68984787
:1067600023791BB9A36B20465B689847F6B286F382
:1067700011882046FFF784FE2046FFF7A5FFCDE7EE
:10678000F8B5002504462F46628CAEB2A38C12B237
:106790001BB29A420BD1628CA38C12B21BB29A42EA
:1067A0001ED01EB32046BDE8F840FFF779BEA36BAC
:1067B0002046DB6A98470028EDD0A38C2046A16ACA
:1067C0001BB2A26BC95C526A9047A38CB4F9262015
:1067D00001331BB29A42A38400DCA7840135D3E7BE
:1067E000A36B002120469B6A9847DAE7F8BD2DE9A4
:1067F000F341C58D4FF00008B0F9323004462DB298
:1068000047460135AB42D8BF0025A36B2046DB6964
:10681000984700282BD0268E36B2AE421CD0A36BF0
:1068200001A920465B699847B4F91430C0B2002B27
:106830002FDAAE42E9D0E38D08F10108626B1BB29A
:106840001FFA88F8D0542BB20135E385B4F9323001
:10685000AB42D8BF0025D8E7A36B1B6A002BDED064
:106860000122B4F93210204698470028D7D0B8F159
:10687000000F02D02046FFF703FE3FB13946B4F9BE
:10688000140001F071FE2046FFF71EFF02B0BDE8C4
:10689000F0812369DB07CCD5032805D01A28C8D19D
:1068A000002F08BF0727B0E70A27AEE708B5044B5B
:1068B000186818B103689B6803B19847002008BDA9
:1068C000800000240020704700230B81406F49683E
:1068D000C388CB8003681B6918477047C36B93F864
:1068E0005430002B0CBF6FF07F00002070477047C2
:1068F00000207047C36B93F85500032894BF002015
:106900000120704770B5036806460D469B6898479E
:10691000044660B1C5802846FDF742FC054620606C
:1069200028B9336821462C463046DB689847204614
:1069300070BD806890F8543013B10121FFF79CBE00
:10694000704700218068FFF797BEF8B50446EFF363
:10695000118500238022EFF3108372B682F3118831
:1069600083F31088C66E8C30FDF7D8FE48B394F8D8
:106970005530A1220227013B84F8553041680B684D
:106980001A7020229F715A7000229A70DA701A7160
:106990005A71DA7194F859705A721F720A23086199
:1069A0003046CB8001230B7133681B69984794F8FC
:1069B0005930EDB203F0030384F8593085F31188A0
:1069C000F8BD6FF00B00F2E72DE9F0470446EFF356
:1069D000118600238022EFF3108372B682F31188B0
:1069E00083F3108800F17C073846FBF7DBFA94F854
:1069F0005D30002B68D094F85B50002D64D104F119
:106A00009409D4F89480B8F1000F4ED0D8F804104F
:106A1000B8F808300A68B1F808A01A44B4F932107E
:106A2000AAEB030AE38D104601331FFA8AFA9BB2E0
:106A30008B42A8BF0023218E851A09B2ADB28B42CA
:106A400019D1228E12B2934206D1B4F9321001222A
:106A50002046013900F06BF815B12046FFF710FD14
:106A6000AA451BD84846FDF759FE41462046FFF788
:106A70002BFF0546C5E7AA45E3D9E58D10F801CB04
:106A8000616B2DB201F805C019B20133E1859BB2EB
:106A9000B4F932108B42A8BF0023CCE7B8F8083015
:106AA0001D44A8F808506FF01B05D4F894302BB1A2
:106AB0002346074AC821384601F0EEFDF6B286F3B8
:106AC00011882846BDE8F0876FF00F05EDE700BF9D
:106AD0002B6B000838B584680869EFF31185002333
:106AE0008022EFF3108372B682F3118883F310884B
:106AF000B1F90A3013F16E0F0CD08BB9038104F198
:106B00009401FDF7EBFD2046FFF75EFFEDB285F344
:106B1000118838BD94F85630013B84F85630F5E7BB
:106B200001462046FFF7D0FEF0E7FFF74DBF38B52E
:106B3000C46B94F8593094F85A1084F85C2003F030
:106B40000205F1B17AB145B123F00203204643F0CA
:106B5000010384F85930FFF7F8FE012384F85B3015
:106B600094F85B0038BD84F85B2035B943F003032B
:106B7000204684F85930FFF7E8FE2046FFF724FF4F
:106B8000EEE7002DECD143F00303204684F85930A2
:106B9000FFF7DBFE84F85B50E2E710B5C06BEFF364
:106BA000118400238022EFF3108372B682F31188E0
:106BB00083F3108859B190F85D3013B9012380F840
:106BC0005D30FFF701FFE4B284F3118810BD80F857
:106BD0005D10F8E72DE9F04F044685B0EFF311831F
:106BE000802702930023EFF3108372B687F3118896
:106BF00083F31088D0F870904FF0000B0397B9F82A
:106C00000630602B38BF60230193D4F88C80B8F134
:106C1000000F26D0D8F804703868EFF3118A039B70
:106C2000EFF3108672B683F3118886F3108801465D
:106C3000B4F822C00D1AA28C0FFA8CFC12B2ADB2BD
:106C4000944516D1618CA28C09B212B2914224D023
:106C500015B12046FFF724FC5FFA8AFA8AF31188FF
:106C60000DBB00209DF8083083F3118805B0BDE806
:106C7000F08F019BAB42E5D9A58CA26A2DB2525D83
:106C800001F8012BA28CB4F92650013212B29542C0
:106C9000A284CDDCA4F824B0CAE7A26B0021204670
:106CA000926A9047D4E704F18C00FDF737FD94F821
:106CB000552039464846013A84F855200122FD8086
:106CC000C7F810803A71D9F800201269904700285F
:106CD0009BD0C7E770B50E4684680869EFF311854D
:106CE00000238022EFF3108372B682F3118883F3BE
:106CF000108804F18C01EDB2FDF7F0FC94F85530EA
:106D0000013384F8553085F31188B6F90A3023B978
:106D10002046BDE87040FFF75DBF70BD41B1C06B5C
:106D2000428C838C12B21BB29A4201D0FFF752BF41
:106D3000704770B583685C6940F20933994200F08E
:106D4000F48029DCB1F5817F00F0828006DC40F21E
:106D5000011399424DD06FF01805A1E040F20733BE
:106D6000994200F0B980B1F5427FF4D1EFF3118080
:106D700000238021EFF3108372B681F3118883F32F
:106D80001088A18C638C09B21BB2994200F3C680B3
:106D9000638CA18C1BB2B3E040F60253994216D02B
:106DA00006DC40F601539942D5D1A266002577E072
:106DB00040F60353994215D040F604539942CAD184
:106DC00084F859202046BDE87040FFF7BEBD002A78
:106DD00000F0CB8054F85E3F1360A3889380A379C2
:106DE0009371E3E7002A00F0C08094F858301360F4
:106DF000DCE7002A00F0B980A3681360E368536001
:106E00002369D36094F8633003B3012B4FF480718E
:106E10000CBF4FF4007300230B4394F8621010462C
:106E2000022943F030030CBF402100210B43936043
:106E300094F85A10002914BF4FF0004100210B4371
:106E40009360D4F85E10FDF73BFEAFE71946E3E729
:106E5000002A00F08A801368A3605368E360D36857
:106E60002361936894F85A20B2EBD37F9ED0002B15
:106E70001ADB94F859309A0714D443F003032046E0
:106E800084F85930FFF761FD05460023204684F859
:106E90005A3084F85B30FFF797FD012384F85D30AA
:106EA000284670BD0025F0E70126002394F85C50C9
:106EB00084F85A6084F85B30002DEED094F8593095
:106EC000204623F00203334384F85930FFF73DFD99
:106ED00084F85B600546E0E7EFF311800023802132
:106EE000EFF3108372B681F3118883F31088218E3B
:106EF000E38D09B21BB2994208DCE38D218E1BB2EF
:106F000009B25B1AC1B281F3118870E7218EE58D59
:106F100009B2B4F932302DB2491BF2E7A18C658C6D
:106F200009B2B4F926302DB2F6E7EFF31180002351
:106F30008021EFF3108372B681F3118883F31088F8
:106F4000618CA38C09B21BB2994206DAA38C618CC6
:106F50001BB209B25B1A013BD4E7618CA58C09B264
:106F6000B4F926302DB2491BF4E76FF0150597E709
:106F700070B50D46044658B151B1086808B1FDF727
:106F800007F9236829462046DB68BDE870401847AA
:106F900070BD10B590F85430044693B1002180F8CC
:106FA0005410FFF769FBE06E03685B689847206F39
:106FB00003685B689847606F0368BDE810405B68D2
:106FC000184710BD70B50E468468EFF31185002395
:106FD0008022EFF3108372B682F3118883F3108856
:106FE00000212046FFF748FB2046FFF7D2FF002391
:106FF000EDB26384A38485F3118833685B6923B1A0
:1070000030460121BDE87040184770BD2DE9F041C0
:1070100084680D46002C49D02046FFF7BAFF322085
:10702000FDF792F8E16E29B12B6828465B68984716
:107030000023E366A16F21B16868FFF799FF002381
:10704000A367264604F130074FF00008D6F8E81091
:1070500021B1606FFFF78CFFC6F8E8800C36BE42A6
:10706000F4D1616F29B12B6828465B6898470023EB
:107070006367EFF3118600238022EFF3108372B66B
:1070800082F3118883F3108804F18C08D4F88C7093
:1070900077B9F6B286F31188216F21B12B682846A3
:1070A0005B689847276700236384A384BDE8F08169
:1070B0004046FDF733FB41680029E7D0206FFFF71A
:1070C00057FF94F85530013B84F85530DEE7FFEC6C
:1070D0002DE9F74F84680D46804621654B684021B5
:1070E0009C606868FFF70EFCA06700287ED0414BCB
:1070F0000122C3602846D4F8B0102B6861F07F01EC
:107100001E680323C9B2B047E06630B96FF01204BD
:1071100029464046FFF77AFF64E084600122D4F8F4
:10712000B41028462B6861F07F011E680223C9B2A3
:10713000B04720670028E9D0846000222B682846E9
:1071400094F8B8101E680223B04760670028DDD0AD
:1071500004F1E40604F58A7A4FF0000B264BB146A1
:1071600084604021606F0193FFF7CCFB70600028C2
:107170003CD0A6F808B006610C3656F8082C019BE6
:107180005645D360EDD104F1C4064FF0800A60216A
:10719000206FFFF7B7FB706040B30661174A736852
:1071A000DA60EFF3118BEFF3108772B68AF3118870
:1071B00087F3108804F18C013046FDF78FFA94F8BC
:1071C00055205FFA8BF3013284F8552083F3118840
:1071D00008364E45DBD12B685C691CB1012128467D
:1071E000A0470024204603B0BDE8F08F6FF00B04E9
:1071F0008EE700BFDB680008D56A0008D56C000880
:1072000037B50446154608461A466946002300F07D
:1072100037FA23682A4669461B682046984703B018
:1072200030BDFFEC2DE9F04190F8543004460E4695
:107230008B4203D100252846BDE8F081FFF7A9FE67
:10724000002EF7D0012E41D1002204F19C07E06E00
:107250003B461146FFF7D4FF051E33DBE36E0022E9
:1072600002219C603B46206FFFF7CAFF051E29DB09
:10727000236F324631469C603B46606FFFF7C0FF8C
:10728000051E1FDB636F264604F13007DFF84480DC
:107290009C60D6F8E810C1F80C80606F03681B6929
:1072A0009847054670B994F856300C360133BE4203
:1072B00084F85630EDD10121204684F85410FFF7B0
:1072C000DBF9B8E72046FFF764FEB4E76FF0150579
:1072D000B1E700BFD56A00082DE9F8438946177960
:1072E000517992F8068047EA0127D179856892F8AA
:1072F00003E048EA01289078117840EA0E2CAE6F3E
:1073000011F060040FFA8CFC40F0828053781FFA71
:107310008CF4063B052B00F2CB80DFE803F003C9B9
:10732000443B664DBEF1020F27D0BEF1030F2DD0B6
:10733000BEF1010F40F0BC80346800F09DF900F10F
:107340001002234650F8041B904243F8041BF9D165
:10735000028812201A8040454FF001033146A8BF31
:1073600040463371F080D9F8040003681B699847E0
:10737000002809DA0023738106E005F19C013068DA
:1073800000F0B6F90028E6DABDE8F883316800F0CD
:1073900037F9F7E7002940F08B805FFA8CF1284637
:1073A000FFF740FFEEE7802940F08280336895F8D0
:1073B00054201A700120CEE7012979D195F8543074
:1073C000012B75D1D5F8A0309F4202D001339F42E6
:1073D0006ED1002C6CD12846FFF7DBFD95F85410D8
:1073E0002846FFF71FFF0020B5E7812960D195F8F7
:1073F0005430002B5CD1D5F8A0309F4202D001332D
:107400009F4252D1002C50D1336883F800C0D1E79D
:10741000202C4DD15278203A032A49D8DFE802F0D7
:1074200012022B3AA12943D1D5F8A0309F423FD177
:1074300055F85E2F072033681A60AA889A80AA79C7
:107440009A7188E7212933D1B8F1070F30D1D5F8E7
:10745000A02097422CD143B11968C5F85E109988D5
:10746000A5F862109B7985F86430AB6E002BBAD01A
:1074700000209847B7E721291AD1D5F8A0309F42BC
:1074800016D10CF0030CAB6E85F858C0002BAAD0B7
:107490000120EEE721290BD1D5F8A0309F4207D17A
:1074A000AB6E002B9FD00220E3E76FF020006BE76C
:1074B0006FF05E0068E770472DE9F04F8FB024222F
:1074C00083468A4605A80021FDF790FA0227042387
:1074D0004FF003094FF0010843F258200497069338
:1074E000CDE90898CDE90A79FCF75AFE044650B96F
:1074F0006FF00B06BAF1000F01D0CAF80040304619
:107500000FB0BDE8F08F43F24C2600210025324633
:10751000FDF76CFA0DF1100E04F19C0C84F857B0D5
:10752000BEE80F00C4E92355C4E92555ACE80F00B7
:10753000BEE80F00ACE80F009EE803004FF44243A2
:107540001E4A8CE80300A4F85E300823A4F860808B
:10755000102184F864304FF4167384F8038004EB30
:107560000608638604F58A7384F859906846A4F87F
:107570006250636342F6E063E38404F55B73A362E5
:107580000F4BC4E90E340F4B88F80470A3515B46CF
:10759000C8F8084001F042FB21466846FEF728FF84
:1075A000061E05DB40464446FCF7CEFB0646A1E737
:1075B00020462C46FCF7ECFD9CE700BF209F00080E
:1075C000489F0008309F000830B585B084680B4A9A
:1075D000102194F857300546684601F01FFB6846B5
:1075E00000F0A0FD2846FCF7C9FB04F17C00FAF787
:1075F000D9FC2046FCF7CCFD05B030BD209F00082B
:1076000070B50C4604282BD8DFE800F01521031DC7
:107610001F00154D2846FDF739FA00231F2819468B
:1076200028BF1F20984214DC4000032302306370FF
:10763000C0B2207006E0032304204B7009230870B9
:107640008B70C87070BD094DE4E7094DE2E7094D44
:10765000E0E704EB4302EE5C01339670D170E1E7A2
:107660006FF01500EEE700BF849F000805A000083A
:107670009C9F00087C9F000800487047A19F00085D
:10768000012810B515D003D3022821D000200FE027
:10769000052307204B700870536963F07F038B70DC
:1076A0000323CB7040230B7100234B710A238B7192
:1076B00010BD072305240B704C70D26988718A7045
:1076C0000222CA7040220A7100224A711846EFE76E
:1076D000072305240B704C709269C87062F07F021A
:1076E0008A7040220A7100224A7101228A71EDE7F4
:1076F0002DE9F0410D460446002800F08B80002162
:1077000004260846FFF7F4FF802302224FF0090EFB
:10771000A07001210012E37114F1090F4FF0FA0378
:1077200084F800E06270E07022716171A6712372CA
:1077300070D0A6724FF0100C84F809E005206B6839
:10774000242784F815C04FF00308E3724FF0060CAD
:107750000023A074E67584F81AC04FF0070CE07699
:1077600084F81E8023736173A273E27321746374BF
:10777000E7742375A17527766276277761776F683E
:1077800084F821000F4484F820C0E7776F6984F8FB
:1077900023804FF00A0867F07F0784F8253084F8CB
:1077A0002270402784F8247084F8268084F827E02B
:1077B00084F828606E6884F82A300E4484F82B2000
:1077C00084F82C8084F8296084F82D3084F82E30D9
:1077D00084F82F3084F830C084F83100EE6984F8E2
:1077E000332084F8326084F8347084F8353084F8BB
:1077F000361084F837C084F83800A86984F83A2035
:1078000060F07F0084F83B7084F83C3084F83900E5
:1078100084F83D103E20BDE8F081002070471046FE
:10782000704708B54AB10B794A7903F00503134351
:107830004B7113B1C86800F02BFE002008BDFFECAF
:1078400000234FF4DB720249024800F04ABC00BF3B
:10785000B49F0008D49F00080846FBF7CDB9FFECA1
:1078600038B50C4615460848254400F097FDAC4253
:1078700004D1054800F00CFE002038BD14F8010BBF
:10788000FBF7BAF9F3E700BF8400002400F034B935
:10789000F8B5837805460F468B4220D289004068B0
:1078A00001F074F8064668B1AC788020FCF788FCDB
:1078B00046F8240070B9013CAB789C4205DA3046AA
:1078C000FCF766FC6FF016000AE056F82400FCF79F
:1078D0005FFCF0E70134BC42E7D36E60AF7000207C
:1078E000F8BD01220021FCF783BFF8B58678054674
:1078F000741EA4003EB96868FCF74AFC2846BDE83F
:10790000F840F9F7D1BD70276B6818593844103F1B
:1079100000F018FA17F1100FF6D16B68013E1859F4
:10792000043CFCF735FCE5E72DE9F84FDDF828B01D
:107930008A4691461F46804600F088FC044600F0C7
:107940005DFD051E3ADB0826A3789BFBF6F6B342E5
:1079500009DC711C2046FFF79BFF051E03DA204659
:1079600000F096FD2AE0DBF10003D4F804E00BF010
:10797000070503F007030EEB860158BF5D42A1EB3C
:107980000E0051F804BB0BEB05129368A2EB0B0C35
:10799000CBB9C2F800A005EBC60562681358634472
:1079A000C3F8049063681B586344C3F80880636895
:1079B0001B5820466344DF6000F06AFD2846BDE89E
:1079C000F88F5E46DBE701351032082DDDD106F178
:1079D000010BA37800255B45F3DCB11C2046FFF7C3
:1079E00057FF051EBBDB63684FEACB0553F82B300E
:1079F000C3F800A0636853F82B30C3F804906368A1
:107A000053F82B30C3F80880636853F82B30DF60DD
:107A1000A5E7F8B5002304460F460B6000F016FCFE
:107A20000646E0B18378B4EBC30F1BD200F0E6FC4E
:107A3000051E12DB082362427168304602F007021D
:107A400094FBF3F304F0070451F8233058BF544279
:107A500003EB04143C6000F01BFD2846F8BD6FF0FA
:107A60000A05FAE76FF00805F7E7F0B585B00446B8
:107A700000F0ECFB054600F0C1FC002814DB002CF4
:107A80000DDBAB78B4EBC30F09DAE2106B6804F0DE
:107A9000070453F8223003EB04139A6832B92846DE
:107AA00000F0F6FC6FF0080005B0F0BD1A466E4617
:107AB00003F110071068083252F8041C3446BA4229
:107AC00003C42646F6D1102200211846FCF78EFF8B
:107AD000284600F0DDFC684600F034F9E4E710B514
:107AE000FFF7C3FF041E05DA6442FCF77CFD046067
:107AF0004FF0FF34204610BD10B5074C0122002185
:107B00002046FCF775FE4FF6FF7363800023A380C9
:107B1000BDE8104000F04CB89814002438B50B4C68
:107B200000F07EFD0546B4F90230834204D1A388FB
:107B300000200133A38038BD204600F05FFC002800
:107B4000A2BF01236580A380F5E700BF981400243D
:107B50000748B0F90430012B02DD013B83807047F8
:107B60004FF6FF7343800023838000F091BC00BF79
:107B70009814002410B50446034613F8012B2AB9C3
:107B8000001B1C30FCF71CFB20B910BD2F2AF7D0BE
:107B90001846F1E700F11803013C14F8012F12B95F
:107BA00000221A70F1E72F2AFAD003F8012BF4E72C
:107BB00008B50348FFF7DEFF024B186008BD00BFA1
:107BC000E49B0008A014002400232DE9F04117468F
:107BD0001360027888B0002A45D08DF81C30CDE9BA
:107BE000010301A8CDE90333CDE9053300F04EF8D8
:107BF000002835DA019EDDE90354304600F036F8FE
:107C0000037880463046D3B1FFF7B4FF48B96FF030
:107C10000B04069808B1FCF7BBFA204608B0BDE893
:107C2000F0813DB16B68C0E90043686000254646BD
:107C30000446E2E7A368C0E90043A060F6E7FFF767
:107C400099FF0028E3D035B16B68C0E90043686054
:107C500038600024DDE7A368C0E90043A060F7E7CF
:107C60006FF01004D5E76FF01504D6E703461A4607
:107C7000184612F8011B31B12F2905D118460133DE
:107C800002782F2AFAD070471346F0E7F8B5036858
:107C900005461A782F2A08D0274A1430274900F0C1
:107CA000B0FF6B69002B40D02B60254B28681C6807
:107CB00003782F2B3CD1002637464CB96FF00103D7
:107CC00022462A61C5E90004C5E902761846F8BDD6
:107CD00004F11701431E11F801CF13F8012FBCF175
:107CE000000F0FD10AB12F2A16D1FFF7BFFF03787B
:107CF000B3B1E38903F00F03032B13D0A368264627
:107D000000240AE022B12F2A02D0944504D3E2D9FC
:107D10006FF001030024D3E7636827461C46CCE7D5
:107D20000246CEE702460023CBE76FF00B03CDE718
:107D30006FF01503CAE700BFE49B0008F49F00083A
:107D4000A014002470B5866805467EB134691CB164
:107D500064680CB1A0470446304600F004FA0023E2
:107D6000C5E90033C5E90233204670BD3446FBE760
:107D700070B5866804460B4615463EB136692EB18D
:107D800036691EB1B04700280DDA70BD012D05D04F
:107D9000022D0AD025B16FF01500F6E76268134492
:107DA000002BF8DB63606068EFE76FF05700ECE7EB
:107DB00037B50C4601A91546FFF72BFE002804DB5A
:107DC0002A4621460198FFF7D3FF03B030BD10B516
:107DD000FFF7EEFF041E05DA6442FCF704FC0460C2
:107DE0004FF0FF34204610BDCB0702D503699B68D6
:107DF0005BB111F0020106D00369DB68002B14BFF0
:107E000000216FF00C01084670476FF00C01FAE793
:107E10002DE9F047074688B090469A46002955D08C
:107E200012F0060F4FF0000501A8019114BF109B3E
:107E30004FF4DB79069518BFD3F800908DF81C50ED
:107E4000CDE90255CDE9045500F07AF9041E2EDB88
:107E5000029EF38903F00D03012B34D1336993B3F0
:107E600041463046FFF7C0FF041E1BDBC7E9008513
:107E7000C7E9026533691C6834B9069800BB002461
:107E8000204608B0BDE8F087F38903F00F03032B09
:107E900013D129EA0A03424605993846A04700282B
:107EA0000446EADA00233046BB6000F05CF906982D
:107EB0000028E5D0FCF76CF9E2E73846A047EEE78A
:107EC000FCF766F9DBE76FF00504EBE76FF01504EC
:107ED000D6E770B5044686B00D46164600F034FE6F
:107EE0002146034600962A4602A8FFF791FF041E8A
:107EF0000CDB002304980093059BDDE90212FFF7D9
:107F000013FD041E02DA02A8FFF71CFF204606B08C
:107F100070BD0EB417B505AA52F8041B0192FFF705
:107F2000D8FF041E05DA6442FCF75DFB04604FF0E5
:107F3000FF34204603B0BDE8104003B0704710B4D2
:107F400004688368E40707D55BB11B694BB19B6884
:107F50003BB15DF8044B18476FF00C005DF8044B23
:107F600070476FF00800F9E737B50C4601A91546D0
:107F7000FFF74FFD002804DB2A4621460198FFF752
:107F8000DEFF03B030BD10B5FFF7EEFF041E05DACB
:107F90006442FCF728FB04604FF0FF34204610BD1C
:107FA00010B40468A40708D583685BB11B694BB1A2
:107FB000DB683BB15DF8044B18476FF00C005DF8CF
:107FC000044B70476FF00800F9E737B515460C46CB
:107FD00059B101A9FFF71DFD002804DB2A462146FF
:107FE0000198FFF7DDFF03B030BD6FF01500FAE731
:107FF00010B5FFF7EAFF041E05DA6442FCF7F3FA56
:1080000004604FF0FF34204610BD2DE9F347B0F176
:108010000008894614461F465BDB12B900F096F94A
:108020000446B8F1020F16DD01A94046FFF7F1FC46
:10803000051E04DB019B986830B96FF00105002F25
:108040003BD000233B6038E04946FFF7CDFE10B13E
:108050006FF00C05F3E7B8F1020FA66834DD482095
:10806000FCF7AEF80446B8B306F1280A504600F013
:1080700095F9051E03DA2046FCF78AF8DFE7D6F803
:108080000831F3B11C60C6F80841504600F000FA10
:108090002046FCF7F1FA04F1200304F14002C4F891
:1080A00004802361E361A4F84090C4E905230C2314
:1080B00084F842309FB100253C60284602B0BDE8FC
:1080C000F087C6F80441DEE7482404FB08642C343A
:1080D000E1E76FF00805B2E76FF00B05AFE73D464B
:1080E000EBE72DE9F34107460E4690461D46FFF7A4
:1080F00015FD041E12DB01AA41463846FFF764FD58
:10810000041E09DB019A0024D38923F00F0343F0F6
:108110000103C2E90465D381FFF71AFD204602B0CE
:10812000BDE8F08138B50546FFF7F8FC041E05DB15
:10813000284600F05DF80446FFF70AFD204638BDEA
:1081400038B50546FFF7EAFC041E0ADB2846FFF7B0
:108150009DFD041EA1BF6A68938901339381FFF7D7
:10816000F7FC204638BD10B50446D0B1FFF7D6FC69
:108170000028FBDBB4F90C300BB1013BA381B4F94F
:108180000C30002B09DCE389DB0606D5FFF7E0FCA9
:108190002046BDE8104000F040B8BDE81040FFF7B1
:1081A000D7BC10BD10B5002488B0F8B10123CDE9CB
:1081B000010401A88DF81C30CDE90344CDE9054444
:1081C000FFF764FDA04207DBDDE90242636852B1BC
:1081D00053600023C4E90033069808B1FBF7D8FFC9
:1081E000204608B010BD049A9360F2E70446F7E712
:1081F00010B5FFF7D7FF68B1B0F90C4034B1C289B0
:1082000042F01002C2816FF00F0010BD00F005F8BF
:108210002046FAE76FF00100F7E710B5044650B1C9
:108220004068FFF7FAFFA068FFF7F7FF2046BDE8B8
:108230001040FBF7ADBF10BD00F08EBB024A1368C3
:1082400001331360704700BFA4140024024B1B6865
:10825000986800B120307047780400240F4B10B5A7
:108260001B680446B3F91E20002A0ADD1A7E037E2D
:108270009A4206D20A49F9F7F3FE01230020A376B9
:1082800010BD06492046F9F7EBFE022320B1032278
:10829000A27622689376F3E7A376F1E778040024C8
:1082A0006C04002438B5436804465BB903680322B4
:1082B00001259A7620460449FCF762FA00232846F5
:1082C000A37638BD0025F5E778040024F0B51349FE
:1082D0000020134C0226032722680B6813B90B6099
:1082E0004B60F0BDD3F800C0B2B193F818E0157E32
:1082F000AE450BD95568C3E900254DB9012053603F
:10830000967623609F761A466346E7E71268EBE7A6
:108310002B6053609E76F6E75368FFDE6C04002402
:1083200078040024024B1B6898682830704700BF0F
:1083300078040024044B1B6823B11868B0FA80F05D
:10834000400970470120704778040024014B1868E9
:10835000704700BF7804002438B50F4B0C461D68E9
:1083600070B1F9F717FCA0B1AB8B03F00303022B3C
:1083700007D0AA6883689A4203D06FF00C0007E028
:108380002846436B2360836B6360C36B0020A3604C
:1083900038BD6FF00100FBE77804002438B5164BB8
:1083A0001C68EFF3118500238022EFF3108372B66F
:1083B00082F3118883F31088D8B103881BB2002B95
:1083C000038803F1FF331BB2038005DD0020206426
:1083D000EDB285F3118838BD0023206405212046C5
:1083E0002384F9F7E3FFB4F920000028F0D04042DD
:1083F000EEE76FF01500EBE77804002410B50446B3
:108400002046FFF7CBFF031DFAD010BD10B5FFF7D4
:10841000C5FF041E06DA6442FCF7E5F804604FF07D
:10842000FF3010BD0020FCE7114B10B51968D8B122
:10843000EFF3118200238024EFF3108372B684F3EC
:10844000118883F3108803881BB2002B09DD038891
:10845000013B1BB2038000200864D3B283F3118870
:1084600010BD6FF00A00F8E76FF01500F8E700BFE5
:108470007804002410B5FFF7D7FF041E05DA644224
:10848000FCF7B1F804604FF0FF34204610BDFFEC5C
:1084900010B500282ED0EFF3118400238022EFF3D3
:1084A000108372B682F3118883F31088038847F62D
:1084B000FF721BB2934205D1E4B284F311886FF0CE
:1084C0008A0010BD038801331BB2038003881BB2EE
:1084D000002B0ADC094B1B683BB11A6C8242FAD1B3
:1084E000002218461A64FAF7E3F8E4B284F311881C
:1084F0000020E6E76FF01500E3E700BF8C040024DE
:1085000010B5FFF7C5FF041E05DA6442FCF76BF8EF
:1085100004604FF0FF34204610BD70B505460C4690
:10852000F8F7CCFCEFF3118600238022EFF31083E1
:1085300072B682F3118883F310882B881A0409D449
:108540002B881B040ED5F6B286F31188F8F7C4FC0D
:10855000002070BD002CF3DD013C2846FFF798FF9A
:1085600024B2EAE72C80EEE737B5051E0C4616DB91
:108570001F2917D8F8F7A2FC0023042269462846D1
:108580008DF800408DF801308DF802200193F9F745
:108590009BF90446F8F7A0FC204603B030BD6FF00D
:1085A0005704F9E76FF01504F6E7FFEC07B568B17B
:1085B000084A0021B0FBF2F302FB130000934FF4D2
:1085C0007A7358430190684600F0E4F803B05DF810
:1085D00004FB00BF40420F0038B50F4C2568284609
:1085E000FFF760FE0D4B1B680BB1FFF76FFE2468B1
:1085F00028460421E38B0133E3830223A376F9F7B2
:1086000005FD0121B5F90C0000F018F80323A3764D
:10861000E38B013BE38338BD780400246C04002421
:10862000054B186838B1837E032B02D1B0F90C00DA
:1086300070476FF0020070477804002470B50E4652
:10864000EFF3118500238022EFF3108372B682F3DB
:10865000118883F31088F9F79DFA0446EDB2A0B1B2
:10866000827E0C4B53F83210FCF78AF885F31188A0
:10867000002120463246F9F731FA217F204601F0E9
:108680000301BDE87040F8F7DBBE85F311886FF099
:10869000020070BD8C9A00082DE9F0410C46164688
:1086A00098460546002839D0002A37D0002935DB06
:1086B000EFF3118700228023EFF3108272B683F369
:1086C000118882F3108843680BB1F9F76BFC1F49DE
:1086D00001346E600E68C5F80C801EB92846FBF7A1
:1086E000FDFF2CE03046334600229968521801D530
:1086F000196831B9A24214DC196829B9A41A1349BE
:10870000ECE718460B46F0E78868024418460B462B
:10871000F0E70E4A294600F023FA10E06FF015004A
:1087200012E099689E42A2EB0102A4EB0204A1EBC5
:1087300004019960EDD10549284600F00AFAAC60C1
:10874000FFB287F311880020BDE8F081F40900240E
:1087500070B50F4C22685AB19368013B002B9360AF
:1087600006DC25460026236813B19B68002B00DD3C
:1087700070BD2846FBF7D2FF23681BB19A68816859
:108780000A449A6043684660C0689847EBE700BFB8
:10879000F40900242DE9F7430F46064600283AD095
:1087A00042681E4B9A4236D8EFF31185002380228F
:1087B000EFF3108372B682F3118883F31088DFF829
:1087C00060806846EDB2D8F80090FCF746F8324673
:1087D0000021684600F036F810F10B0F044606D170
:1087E00085F311880024204603B0BDE8F0837FB1F3
:1087F00001A9304600F0D0F9D8F800300198394688
:10880000A3EB090398428CBFC01A002000F0B6F910
:1088100085F31188E7E76FF01504E4E7FFC99A3B99
:10882000A4140024827E062A0AD140F2FF22A0F876
:108830005C20742280F85E2000220266F9F738BFBF
:108840007047FFEC3C4B2DE9F74F80460D469146B3
:108850001C68EFF3118700238022EFF3108372B6B8
:1088600082F3118883F3108806682046F9F712FB1B
:108870003040FFB20190B0B101A8F8F7E9FE01461F
:108880002046F8F793FE2DB1024652F8043F2B60C4
:1088900053686B600679F8F7ADFE87F311883046B0
:1088A00003B0BDE8F08FD8F80030A364B9F1000F31
:1088B00036D0D9F804300021204804F12406D9F834
:1088C00000E010EB030ADFF880C01D4A41EBE37BB8
:1088D000504600235946ECFB0E0100F0B3FA234644
:1088E0000146184A3046FFF7D7FE20460621F9F721
:1088F0005DFD3046F9F756FB94F85C1000231F2904
:10890000A36412D84046FBF7ACFF88B194F85C60D2
:10891000002DC2D054F85C3F2B6063686B60BCE7ED
:1089200006212046F9F742FDE6E76FF00A06EFE779
:108930006FF00306ECE700BF780400243F420F000D
:1089400040420F002588000800CA9A3B08B500F095
:108950001BFA002008BDFFEC08B5084A0F20084BA1
:1089600008491A6000225A60F8F750FA064B0722AD
:108970000F201A60BDE80840F7F7E0BFFF5207007C
:1089800014E000E04D89000810E000E0024B0A46C8
:108990000146186800F002B86C0F00242DE9F84F6A
:1089A000814692460F4621B91146BDE8F84FFBF7C4
:1089B00012BD12B9FBF7B1FC17E0173222F00F0B12
:1089C000DA4500F2B880A1F10804FBF75CFC57F827
:1089D000085CAB450CD804D25A4621464846FBF702
:1089E000CFFDBA464846FBF76EFC5046BDE8F88F0F
:1089F00057F8041C04EB050821F00041D8F80430B6
:108A0000611A002B4B68B4BF00266659002B06EB99
:108A10000503ACBFD1F800C04FF0000C63445B45C8
:108A200077D3ABEB0502BCF1000F52D0B44501D9AE
:108A3000002E50D1944580F08180A2EB0C0A624652
:108A4000D1E902039860886808B1CB68C360944597
:108A5000A4EB020446D90B689B1A2A440B602260DF
:108A6000086840F0004060604846D8F8043003F0E1
:108A700000431A43C8F80420FBF727FC04F108035D
:108A8000A5F1080239461846F7F7AAFF2568BAF19A
:108A9000000F3CD05246074608EB0600D8E9021307
:108AA0009960D8F8081011B1D8F80C30CB60154493
:108AB0009642256025D9B61A6119665123684B6024
:108AC000436803F000431E4346604846FBF7FDFB46
:108AD00087E7002E85D0002A83D09642DCD2921BF5
:108AE000B246ADE72368EA18636843F000432260AA
:108AF0006360D8F8043003F000431343C8F804302F
:108B0000BCE7436803F000432B43436069E7074633
:108B100067E74846FBF7D7FB51464846FBF75BFC47
:108B2000824600283FF461AF39462A46F7F758FFDE
:108B3000394648463EE74FF0000A56E7002A3FF420
:108B400050AF4FF0000A7BE708B500F017F9406816
:108B500008BD0B6803600B6803B948600860704784
:108B600003460846116811B15168994202D1114675
:108B7000FBF7B4BD1A680260186070474FF47A7250
:108B800090FBF2F30B6002FB130302484343002007
:108B90004B60704740420F002DE9D84842680C46B0
:108BA000006800270949D317094EE1FB00239346CB
:108BB0009C46084A1BEB06004FF000034CEB0701F4
:108BC00000F0F0F820600020BDE8D88800CA9A3B89
:108BD0003F420F0040420F0028B121B1038800201E
:108BE0001BB20B6070476FF015007047081E07D06E
:108BF00004DB022802DC6FF0570070476FF01500AD
:108C000070470EB403B503AA52F8041B019200F09A
:108C10001CF802B05DF804EB03B070470CB47FB5EC
:108C20000A4671B1014601A800F042F809AA089964
:108C300001A80092FBF77EFF07B05DF804EB02B0DD
:108C4000704701A800F048F8F0E7F0B58BB0144683
:108C50000E46074602A8019200F03EF82246314631
:108C600002A8FBF767FF049C01342046FBF798FA43
:108C7000054660B10146224605A800F019F8019AA0
:108C8000314605A8FBF756FF3D600BB0F0BD4FF035
:108C9000FF30FAE783680269934207D2C268D15471
:108CA00000218368C26801338360D1547047FFECB0
:108CB000054B013A0360054B026143600023C0E9A4
:108CC00002310B70704700BF958C0008314B0008D3
:108CD0008368013383607047034B0360034B436039
:108CE00000238360704700BFD18C0008314B00081F
:108CF00038B50546FBF7CAFE0130FBF751FA0446CA
:108D000010B12946FBF7BAFE204638BD014A00F0F3
:108D100003B800BFA81400242DE9F0418846174687
:108D20000446C0B125462C4615F8011BD1B140467A
:108D300000F01AF80028F6D129782E46013539B10D
:108D4000404600F011F80028F6D0002333702E467C
:108D50002FB13E6003E012B11468002CE2D120462E
:108D6000BDE8F0810C46FAE70278034601308A42FA
:108D700002D0002AF8D113461846704708B5FBF711
:108D8000C1FE006808BDFFEC08B5054B0BB1FFF74D
:108D900055FAFFF7DDFCBDE80840F7F73CBF00BF20
:108DA0003D8200087BB972B90029BEBF00204FF098
:108DB000004106E008BF00281CBF6FF000414FF0E3
:108DC000FF3000F0E7B9ADF1080C6DE904CE0029E1
:108DD00009DB002B1ADB00F077F8DDF804E0DDE9B1
:108DE000022304B07047404261EB4101002B1BDBC2
:108DF00000F06AF8DDF804E0DDE9022304B0404247
:108E000061EB4101524263EB43037047524263EB13
:108E1000430300F059F8DDF804E0DDE9022304B073
:108E2000404261EB41017047524263EB430300F063
:108E30004BF8DDF804E0DDE9022304B0524263EBB5
:108E40004303704753B94AB9002908BF00281CBF23
:108E50004FF0FF314FF0FF3000F09CB9ADF1080C3E
:108E60006DE904CE00F030F8DDF804E0DDE902231E
:108E700004B07047FFECC2929FED0F6B41EC170BF3
:108E80009FED0F5B27EE066BBCEEC66B4DF804BD85
:108E9000B8EE464BA4EE457BBCEEC77B4FF0000B13
:108EA00017EE103A16EE101A4BEA03005DF804BBF9
:108EB000704700BFAFF30080000000000000F03DED
:108EC000000000000000F0412DE9F047089E044634
:108ED0008846002B4BD18A42154667D9B2FA82F2F6
:108EE0004AB1C2F1200701FA02F320FA07F79540D0
:108EF00047EA030894404FEA154E230CB8FBFEF7EF
:108F00001FFA85FC0EFB178843EA084307FB0CF1A8
:108F1000994209D9EB1807F1FF3080F01B81994283
:108F200040F21881023F2B445B1AA4B2B3FBFEF05F
:108F30000EFB103344EA034400FB0CFCA44509D9A2
:108F40002C1900F1FF3380F00781A44540F2048121
:108F500002382C4440EA0740A4EB0C0400271EB161
:108F6000D4400023C6E900433946BDE8F0878B4270
:108F700009D9002E00F0EB800027C6E90001384631
:108F80003946BDE8F087B3FA83F7002F47D18B420B
:108F900002D3824200F2FA80841A61EB03030120BB
:108FA0009846002EE0D0C6E90048DDE702B9FFDEB2
:108FB000B2FA82F2002A40F08F80491B4FEA154E28
:108FC0001FFA85F80127B1FBFEFC230C0EFB1C11D8
:108FD00043EA014308FB0CF1994207D9EB180CF165
:108FE000FF3002D2994200F2CD808446591AA3B2D2
:108FF000B1FBFEF00EFB101443EA044408FB00F83A
:10900000A04507D92C1900F1FF3302D2A04500F288
:10901000B6801846A4EB080440EA0C409FE7C7F16D
:10902000200CBB4022FA0CFE4EEA030E01FA07F4B4
:1090300020FA0CF521FA0CF34FEA1E482543B3FB46
:10904000F8F92C0C08FB19331FFA8EFA44EA034393
:1090500009FB0AF49C4202FA07F200FA07F10BD965
:109060001EEB030309F1FF3080F087809C4240F241
:109070008480A9F1020973441B1BADB2B3FBF8F065
:1090800008FB103345EA034400FB0AFAA24508D95D
:109090001EEB040400F1FF336BD2A24569D90238FC
:1090A000744440EA0940A0FB0289A4EB0A044C4541
:1090B000C2464B4654D351D0002E69D0B1EB0A05BD
:1090C00064EB030404FA0CFCFD40FC404CEA05058B
:1090D000C6E90054002747E7C2F1200320FA03F74E
:1090E000954001FA02F021FA03F34FEA154E384396
:1090F000010CB3FBFEF71FFA85F80EFB173341EAAC
:10910000034107FB08F38B4204FA02F407D96918FC
:1091100007F1FF3C2FD28B422DD9023F2944CB1AB5
:1091200081B2B3FBFEF00EFB103341EA034100FBBA
:1091300008F38B4207D9691800F1FF3C17D28B4224
:1091400015D902382944C91A40EA07473BE7374690
:10915000304609E70746E7E61846FBE64145ABD24D
:10916000B8EB020A69EB0E0201381346A4E7604629
:10917000E9E7184695E76746D1E781467CE702387C
:109180002C4447E7ACF1020C2B442FE7384608E7A4
:109190003746E9E6704700BF0720704710B5082042
:1091A000064CF8F7D1FF4FF0006322202360F8F758
:1091B000CBFF0023024A2360136010BD8044025895
:1091C000D844025808B5042000F088F9064B4FF443
:1091D0007A70DB68584300F075F900F0A5F9BDE836
:1091E000084000F08BB900BF8600002408B500F0ED
:1091F000A3F900F08BF9002000F070F90020BDE821
:10920000084000F05FB9FFEC0C4B1A6842F0010215
:109210001A601A685207FCD5094A002111601A68C1
:10922000084922F0A85222F410221A60064A11605E
:109230001A6822F480221A60704700BF0044025866
:10924000104402580000FF012C44025808B54FF0AA
:10925000006000F012FA4FF00160BDE8084000F035
:109260000CBA08B500F074FB4FF0006000F0F2F9A2
:109270004FF00160BDE8084000F0ECB900F0A6BA7C
:10928000014B1860704700BF08ED00E00E2894BF46
:109290004FF4003000207047431E0D2B10B50446DC
:1092A00007D800F011FA20B12046BDE8104000F0C8
:1092B00020BA10BD00F1006000F5003000F066BB80
:1092C000830705D100F1006000F5003000F09EBB7F
:1092D0000020704700207047014B1868704700BF9E
:1092E0000010005C224BF0B5224C1B682588C3F3AC
:1092F0000B0766681B0C227AAF422BD0A589AF42C0
:1093000005D101220C2505FB02446668227A41F250
:109310000304A34220D042F20104A3421ED042F231
:109320000304A3421CD041F20104A34208BF5A2205
:10933000451E013E0B460D44AB4217D216F8010FF5
:109340005C1C78B92C20A542187001D99C1C5A705D
:10935000601AF0BD0022D5E75922E9E75822E7E775
:109360005622E5E704F8010C2346E5E71C46EFE743
:109370000010005C98000024014BC058704700BFEB
:1093800000E8F11F012803D100210248F8F7C8BE08
:10939000704700BF220B04000128014602D1024899
:1093A000F8F7BEBE704700BF220B0400012808B5C5
:1093B0000AD10648F8F7B4FF80F001010348C9B2AA
:1093C000BDE80840F8F7ACBE08BD00BF220B0400A2
:1093D000D0E9003283F308881047FEE72F4A4FF4A4
:1093E0000030F8B5136800242D4D43F4700313606A
:1093F0001C222C4B1C725C729A72DC72F8F7A4FE71
:109400002948F8F7A1FE0120F7F74AF920462E680F
:10941000F7F746F9254B9E423CD101202746F7F746
:109420003FF92C602046F7F73BF9214800F0EEFAAF
:109430000646204800F0EAFA1F4B98420ED126F06B
:10944000FF021E4B9A4209D1F6B21E2E06D84FF4E7
:109450007A7300275E43B44238BF34460820F8F7D9
:109460005FFF064658B957B1FCF774F90120F7F7CA
:1094700017F90E4B344630462B60F7F711F90221ED
:109480000F48FCF721F920460024FCF7B5F9FCF75A
:1094900061F9F8E740F6B8340127C6E788ED00E047
:1094A0005040005886000024220B040007B007B08B
:1094B000A0010208A40102085D7D05C500ECC2926E
:1094C000FA9F0008034B1B685843034B20F07F4072
:1094D00018607047B000002414E000E000280CBFC2
:1094E00008220122034B04211A6000F00402024802
:1094F000F7F704B9B000002410E000E001220021D9
:109500000148F7F7FBB800BF10E000E008B5002203
:1095100001210348F7F7F2F8024B00221A6008BD58
:1095200010E000E018E000E0022200210148F7F717
:10953000E5B800BF10E000E0002202210148F7F783
:10954000DDB800BF10E000E0042838B505460C4641
:1095500013D80120F7F766F8032D094B4FF00000F0
:109560000CBF24F0FF01002153F825301943054BAF
:109570001960F7F757F8002038BD4FF0FF30FBE7D0
:1095800024A00008504000580128044608B502D124
:109590000021FFF7D9FF2046F7F734FB00F000F871
:1095A0000449054B0A6802F4E06213430B60BFF301
:1095B0004F8FFEE70CED00E00400FA05436803F16D
:1095C00010010A68D207FCD4DA68D20705D5034A2D
:1095D0005A6002F1883243685A6070472301674538
:1095E000084B9A6882420AD802F50012824206D9D4
:1095F000054A916881428CBF18461046704700208A
:10960000704700BFB4000024C800002410B4144602
:1096100040681A46084421465DF8044BF7F76EB8D7
:10962000012300220C21FFF7F1BFFFEC38B50546FE
:10963000BFF34F8F064C6B68186910F0070006D017
:109640000120F7F770F8013CF5D16FF00F0038BD3D
:10965000404B4C0038B5FFF7C3FF054650B1FEF74D
:10966000CDFE041E04DB2846FFF7A8FFFEF710FF1F
:10967000204638BD6FF01204FAE738B5FFF7B0FFA7
:10968000054658B1FEF7BAFE041E05DB2846FFF773
:10969000C7FF2846FEF7FCFE204638BD6FF01204D7
:1096A000FAE7B0F5803F10B504460AD200F5800015
:1096B0004001FFF795FF03698068E41A00EB44104E
:1096C00010BD4FF0FF30FBE7B0F5803F08B50DD27D
:1096D000FFF7E7FF002300F1200201780130FF29A6
:1096E00018BF01338242F8D1184608BD6FF00D0053
:1096F000FBE7F8B50F2800F5806504464FEA4545BD
:109700005ED82846FFF76CFF0646FEF777FE002876
:1097100049DB3046FFF78AFF0746002847D130462D
:10972000FFF74CFF04233A460C21FFF76FFFF36865
:109730004FF470620C21E31A30461B0203F4E0631D
:10974000FFF764FF80233A460C213046FFF75EFFA7
:109750003046FFF76BFF044630BB034604220C2162
:109760003046FFF753FF23464FF470620C2130461A
:10977000FFF74CFF3046FFF753FF3046FEF788FEF9
:109780000CBB2846FFF72CFFE8B105F50036304644
:10979000FFF726FFB8B1B5420CD1002C14BF6FF013
:1097A00004004FF40030F8BD6FF00404E2E76FF0FE
:1097B0000404E2E72B680435013318BF0134EAE7FB
:1097C0006FF00D00EFE76FF00400ECE72DE9F84FC4
:1097D00080460C461646FFF703FF0546002800F0BA
:1097E000B0808368434500F2AC8006EB080203F5C5
:1097F00080139A4200F2A580FEF700FE002856DB97
:109800002846FFF713FF0746002840F097802846B8
:1098100026F01F09FFF7D2FE30230C21A1441A467F
:10982000A8EB040BFFF7F2FE3A46274602230C2171
:109830002846FFF7EBFE4F4523D007EB0B03BFF3A2
:109840004F8FBFF36F8F3A6847F80B207A685A60E2
:10985000BA689A60FA68DA603A691A617A695A6194
:10986000BA699A61FA69DA61BFF34F8FBFF36F8FFC
:109870002846FFF7DBFEF0B96B681B6913F0C06F79
:1098800017D0002302220C212846FFF7BFFE4FF01D
:10989000FF33002214212846FFF7B8FE2846FFF7C1
:1098A000BFFE002E44D12846FEF7F2FD3046BDE84B
:1098B000F88F2037BFE76FF00406EFE74FF0FF3374
:1098C000002214212846FFF7A1FE54F8082023683F
:1098D00004EB08079A422ED17A6863689A422AD12B
:1098E000BA68A3689A4226D1FA68E3689A4222D1FC
:1098F0003A6923699A421ED17A6963699A421AD1F8
:10990000BA69A3699A4216D1FA69E3699A4212D1F7
:109910006B681B6913F0C06F0DD120344C45CDD15D
:109920004FF0FF33002214212846FFF76FFEBAE7FD
:10993000A8EB0408F2E76FF00406F1E76FF0040605
:10994000B1E76FF00D00B2E72822FF21FBF74EB818
:1099500010B5054C2046FFF7F7FF04F12800FFF78C
:10996000F3FF024B636010BDAC140024000002083A
:10997000014610B551F8084B40680134A400224656
:10998000FFF77CFC844208BF002010BD1D4A20F078
:109990001F0310B554689C4225D0D46AA34224D139
:1099A0000123282404FB0323C0F3820413B93CBB26
:1099B000154BD062A01C934243F820101FD1F4B97C
:1099C0001A68072A1BD19A6A013210D003F12804C1
:1099D0002046FFF7CDFF50B120464FF0FF34FFF790
:1099E000B3FF204610BD0023DBE70023DCE705487A
:1099F000FFF7BEFF04460348FFF7A6FFF1E71C6030
:109A00000024EEE7AC140024D414002438B5144B21
:109A100020F01F020568596891421AD0D96A8A421B
:109A200015D101222824C0F382000A2104FB02344C
:109A300001FB02029C4202F1020253F8225006D0BE
:109A4000072804D12046FFF793FF20B1ED432846B5
:109A500038BD0022E6E72046FFF776FFF7E700BFB4
:109A6000AC140024EA17002461726D76372D6D2F37
:109A700061726D5F686172646661756C742E6300FB
:109A800049646C65205461736B00FFEC00000000BA
:109A9000000000006C040024010000007804002491
:109AA000050000007804002405000000580400248C
:109AB000000000008C040024010000009404002435
:109AC0000000000084040024000000004170704287
:109AD00072696E67557000696E6974006972712FE2
:109AE0006972715F756E65787065637465646973BA
:109AF000722E63003C6E6F6E616D653E00FFECC2BE
:109B000001000000C119000802000000C11900088E
:109B100003000000C119000806010000A519000893
:109B200007000000A519000808010000A31900089B
:109B30000A000000C119000809010000C11900084D
:109B40000B000000C11900080C000000C11900083A
:109B50000D000000C1190008736572636F6E3A3A18
:109B6000204552524F523A20416C7265616479200F
:109B7000636F6E6E65637465640A00736572636F0C
:109B80006E3A205265676973746572696E67204327
:109B900044432F41434D2073657269616C206472A8
:109BA000697665720A00736572636F6E3A2045527A
:109BB000524F523A204661696C656420746F20638D
:109BC000726561746520746865204344432F414386
:109BD0004D2073657269616C206465766963653ACE
:109BE0002025640A00736572636F6E3A20537563B3
:109BF0006365737366756C6C7920726567697374DD
:109C00006572656420746865204344432F41434D69
:109C10002073657269616C206472697665720A00EE
:109C2000000002580004025800080258000C0258B4
:109C3000001002580000000000000000001C025844
:109C40002F6465762F747479537800FF000000004C
:109C500000000000000000240000000000000000E0
:109C6000000000000000000000000000B52A00080D
:109C70004D2B0008292A00080B2A00084B29000850
:109C800095280008AF280008E92800084D2A000898
:109C9000F528000809290008FD280008FD2800080B
:109CA000912D0008FF2D0008392E0008552F0008BF
:109CB000492E0008552E000800000000352D000830
:109CC000853200083B2F0008352F0008FD310008C1
:109CD0000B2F000801340008556D656D00FFECC2C4
:109CE0000000000000000000320000000100000041
:109CF0004B000000020000006E00000003000000A6
:109D0000860000000400000096000000050000002E
:109D1000C8000000060000002C0100000700000041
:109D20005802000008000000B00400000900000014
:109D3000080700000A000000600900000B00000096
:109D4000C01200000C000000802500000D00000083
:109D5000004B00000E000000009600000F00000005
:109D600000E100000110000000C20100021000002C
:109D70000084030003100000000807000410000026
:109D800020A107000510000000CA0800061000000E
:109D900000100E000710000040420F0008100000E5
:109DA000009411000910000060E316000A10000082
:109DB00080841E000B100000A02526000C1000005F
:109DC000C0C62D000D100000E06735000E10000029
:109DD00000093D000F100000286E756C6C290069A9
:109DE0006E66006E616E00FF0080E03779C331431C
:109DF00000003426F56BFC420000901EC4BCC64235
:109E0000000040E59C309242000000A2941A5D429E
:109E1000000000E876482742000000205FA0F241E1
:109E20000000000065CDBD410000000084D78741DF
:109E300000000000D01253410000000080841E4149
:109E400000000000006AE840000000000088B34005
:109E50000000000000407F4000000000000049407A
:109E600000000000000014409A9999999999B93F0F
:109E70007B14AE47E17A843F2D431CEBE2361A3F58
:109E80003A8C30E28E79453EBC89D897B2D29C3C60
:109E900033A7A8D523F649393DA7F444FD0FA532D1
:109EA0009D978CCF08BA5B25436FAC642806C80A1F
:109EB00000000000000024400000000000005940A5
:109EC000000000000088C3400000000084D79741D4
:109ED0000080E03779C34143176E05B5B5B89346A6
:109EE000F5F93FE9034F384D321D30F94877825A72
:109EF0003CBF737FDD4F1575050000002C00FFECA3
:109F00006760000801670008095F0008CD6200086B
:109F100000000000C1640008376100080000000074
:109F20002F6465762F74747941434D256400FFECEE
:109F3000D17000080D700008D9720008C56F0008C4
:109F40004369000833690008DD680008EF6800080D
:109F5000F1680008B7740008336D000800000000C5
:109F60009B6B0008000000002F6B00080000000041
:109F70001D6D000800000000F5680008486F6C794E
:109F800062726F0050583420424C20486F6C7962E6
:109F9000726F204B616B75746548370042756C6B4E
:109FA0000012010002020000406231500001010174
:109FB000020301FF00000000000000001B78000801
:109FC0001F7800080000000000000000237800084F
:109FD000000000002F6465762F6E756C6C00FFEC3E
:109FE00059780008597800080000000061780008DE
:109FF0000000000025732F2573002F6465762F74F1
:10A00000747941434D300053544D33323F3F3F3F0D
:10A010003F3F3F0053544D333248375B347C355D0E
:10A020007800FFEC0000000007B007B0020007B0A6
:08A03000000008B0263A09B057
:08A0380090EEFF7F0100000023
:10A040000000000000000000000000000000000010
:10A050000000000000000000000000000000000000
:10A060000000000000002C01580C0024000000003B
:10A0700000005802000A00246C9C00080000002424
:10A0800000000000000000000000000000000000D0
:10A0900000000000000300080000000000C20100F2
:10A0A00037000000000E270700480040387C0900F8
:10A0B000397C090000000000FFFFFFFFE09F00085F
:10A0C0007C000024010018040000000000000000D3
:10A0D0000000E001000000000000000007A00008F0
:10A0E0003F0000005004000014A000083F000000E2
:10A0F00001000000010000000020005200000008E4
:10A1000000000000000000000100000000210052DB
:0CA11000000010080800000000800000A3
:0400000508000000EF
:00000001FF
